:020000040000FA
:100000000C94E2010C940A020C940A020C94721DE6
:100010000C94721D0C94721D0C940A020C940A022A
:100020000C940A020C940A020C940A020C940A0220
:100030000C940A020C940A020C940A020C940A0210
:100040000C94281D0C940A020C94F61C0C94D01CE1
:100050000C940A020C940A020C940A020C940A02F0
:100060000C94EA1D0C940A0207634236B79BD8A78A
:100070001A39685618AEBAAB558C1D3CB7CC5763CD
:10008000BD6DEDFD753EF6177231BF000000803F7B
:1000900008000000BE922449123EABAAAA2ABECD97
:1000A000CCCC4C3E00000080BEABAAAAAA3E000009
:1000B0000000BF000000803F000000000008417801
:1000C000D3BB4387D1133D190E3CC3BD4282AD2B38
:1000D0003E68EC8276BED98FE1A93E4C80EFFFBE30
:1000E00001C4FF7F3F00000000004E414E494E49D1
:1000F0005459494E46CDCCCC3D0AD7233C17B7D1F5
:100100003877CC2B329595E6241FB14F0A0000209A
:10011000410000C84200401C4620BCBE4CCA1B0E19
:100120005AAEC59D7400407A10F35A00A0724E1862
:10013000090010A5D4E80000E87648170000E40B99
:1001400054020000CA9A3B000000E1F5050000805F
:10015000969800000040420F000000A086010000B9
:1001600000102700000000E8030000000064000009
:100170000000000A00000000000100000000002C48
:1001800076D888DC674F0823DFC1DFAE59E1B1B70D
:1001900096E5E3E453C63AE651997696E8E6C284DA
:1001A00026EB898C9B62ED407C6FFCEFBC9C9F40F2
:1001B000F2BAA56FA5F490055A2AF75C936B6CF917
:1001C000676DC11BFCE0E40D47FEF520E6B500D0ED
:1001D000ED902E0300943577050080841E08000002
:1001E000204E0A000000C80C333333330F986E12D0
:1001F000831141EF8D2114893BE65516CFFEE6DBD6
:1002000018D1844B381BF77C1D901DA4BBE424201F
:100210003284725E228100C9F124ECA1E53D2754AD
:100220003D004E6F20445320546865726D6F6D65BC
:10023000746572210020572F6D5E3220555620497B
:100240006E74656E73697479002353656E736F7293
:10025000206572726F722100234E6F20504D207303
:10026000656E736F7221004E6F2073656E736F72CF
:1002700021004C6967687420496E74656E736974F7
:100280007900495220466C616D65204C6576656C3D
:100290003D00476173206C6576656C3D0023496EB7
:1002A00076616C6964206B65792100005EBCE26157
:1002B0003FDD83C29C7E20A3FD1F41009D23BE46DF
:1002C000DB65F88C11AF32CA57E9740000000024D6
:1002D0000027002A0023626D70206661696C6564E6
:1002E000002357656C636F6D6520746F20757365AF
:1002F000204E616E6F204C6F67676572004D533DF5
:1003000000235556207A65726F20766F6C74616792
:1003100065203D00503D0042543D004448543D009E
:10032000234475726174696F6E3D0054494D4544B4
:100330003D0023496E74657276616C3D0054494DF1
:1003400045493D0053484F57533D004C6F67676523
:1003500072204E616D653A20004C4F474745520070
:1003600056455253494F4E005245424F4F5400009C
:100370000000080002010000030407000000000064
:1003800000000000000000230026002900000000FB
:1003900000250028002B00040404040404040402C3
:1003A0000202020202030303030303010204081012
:1003B00020408001020408102001020408102000DF
:1003C000091F4F2711241FBECFEFD8E0DEBFCDBFDE
:1003D00012E0A0E0B1E0ECE3F8E602C005900D9277
:1003E000AE32B107D9F724E0AEE2B2E001C01D920F
:1003F000A13CB207E1F711E0C1EED1E004C02197C2
:10040000FE010E94F431C03ED107C9F70E946B2063
:100410000C9411340C940000089508950895AF923F
:10042000BF92CF92DF92EF92FF920F931F93CF93E1
:10043000DF936C017B018B01040F151FEB015E0143
:10044000AE18BF08C017D10759F06991D601ED91D8
:10045000FC910190F081E02DC6010995892B79F777
:10046000C501DF91CF911F910F91FF90EF90DF9029
:10047000CF90BF90AF900895CF93DF93FC0144815C
:1004800055816081718181E493E00E940F02EC014B
:1004900042E050E069E571E081E493E00E940F02E0
:1004A0008C0F9D1FDF91CF910895FC01538D448DDA
:1004B000252F30E0842F90E0821B930B541710F00F
:1004C000CF96089501970895FC01918D828D98171C
:1004D00061F0A28DAE0FBF2FB11D5D968C91928DF4
:1004E0009F5F9F73928F90E008958FEF9FEF089525
:1004F000FC01918D828D981731F0828DE80FF11DEE
:10050000858D90E008958FEF9FEF0895FC01918D08
:10051000228D892F90E0805C9F4F821B91098F7301
:100520009927089581E493E00E94860221E0892BB7
:1005300009F420E0822F089580E090E0892B29F0D3
:100540000E94920281110C9400000895FC01A48D78
:10055000A80FB92FB11DA35ABF4F2C91848D90E0E5
:1005600001968F739927848FA689B7892C93A089C8
:10057000B1898C91837080648C93938D848D981352
:1005800006C00288F389E02D80818F7D80830895E5
:10059000EF92FF920F931F93CF93DF93EC0181E0D3
:1005A000888F9B8D8C8D98131AC0E889F98980817A
:1005B00085FF15C09FB7F894EE89FF896083E889AD
:1005C000F98980818370806480839FBF81E090E09F
:1005D000DF91CF911F910F91FF90EF900895F62E2C
:1005E0000B8D10E00F5F1F4F0F731127E02E8C8DC6
:1005F0008E110CC00FB607FCFACFE889F98980810B
:1006000085FFF5CFCE010E94A602F1CFEB8DEC0F56
:10061000FD2FF11DE35AFF4FF0829FB7F8940B8F27
:10062000EA89FB8980818062CFCFCF93DF93EC0191
:10063000888D8823B9F0AA89BB89E889F9898C91CA
:1006400085FD03C0808186FD0DC00FB607FCF7CF86
:100650008C9185FFF2CF808185FFEDCFCE010E9486
:10066000A602E9CFDF91CF910895833081F028F47D
:10067000813099F08230A9F008958730A9F0883050
:10068000C9F08430B1F4809180008F7D03C08091E7
:1006900080008F7780938000089584B58F7784BD24
:1006A000089584B58F7DFBCF8091B0008F778093C4
:1006B000B00008958091B0008F7DF9CFCF93DF9384
:1006C000EEE7F3E08491EAEBF3E0D491E6EAF3E0BD
:1006D000C491CC23A1F081110E943503EC2FF0E0EE
:1006E000EE0FFF1FED57FC4FA591B491EC91ED2358
:1006F00081E090E009F480E0DF91CF91089580E0FF
:1007000090E0FACF1F93CF93DF93282F30E0F901C9
:10071000E159FC4F8491F901E555FC4FD491F90161
:10072000E956FC4FC491CC23A9F0162F81110E94E9
:100730003503EC2FF0E0EE0FFF1FE357FC4FA591C0
:10074000B4918FB7F894EC91111108C0D095DE23C5
:10075000DC938FBFDF91CF911F910895DE2BF8CFEF
:10076000CF93DF9390E0FC01E555FC4F249189562F
:100770009C4FFC0184918823D1F090E0880F991F51
:10078000FC01E553FD4FA591B491FC01E357FC4FEB
:10079000C591D49161110EC09FB7F8948C91E22F4E
:1007A000E0958E238C932881E223E8839FBFDF911D
:1007B000CF9108958FB7F894EC91E22BEC938FBF13
:1007C000F6CF8E3008F08E502091000190E4299FE2
:1007D000900111248770822B80937C0080917A0095
:1007E000806480937A0080917A0086FDFCCF8091AE
:1007F00078009091790008953FB7F8948091B702FE
:100800009091B802A091B902B091BA0226B5A89B06
:1008100005C02F3F19F00196A11DB11D3FBFBA2F92
:10082000A92F982F8827BC01CD01620F711D811D52
:10083000911D42E0660F771F881F991F4A95D1F7D7
:1008400008958F929F92AF92BF92CF92DF92EF92D4
:10085000FF926B017C010E94FC034B015C01C114FF
:10086000D104E104F104B9F00E94FC03681979098C
:100870008A099B09683E73408105910580F321E058
:10088000C21AD108E108F10888EE880E83E0981EAC
:10089000A11CB11CE4CFFF90EF90DF90CF90BF90F0
:1008A000AF909F908F9008958F929F92AF92BF923A
:1008B000EF92FF921F93CF93DF93C82F1092B5044E
:1008C0001092B6041092B7041092B8041092B904B2
:1008D00061E08FE00E94B00360E08FE00E9482033D
:1008E0006C2F70E090E080E00E94210460E08FE0D7
:1008F0000E94B0038BE990E00197F1F7C0E9D1E0E5
:100900000E945E03892B71F42197D1F78EEF9FEF40
:10091000DF91CF911F91FF90EF90BF90AF909F908C
:100920008F900895C0E9D1E00E945E03019719F409
:100930002197D1F7EBCFD8E2C0E810E090E9E92E9B
:10094000FF24F3940E945E03892B29F481E0E81AC6
:10095000F108C1F7DBCF0E94FC034B015C0180E989
:10096000E82EFF24F3940E945E03019729F481E0AE
:10097000E81AF108C1F7CACF0E94FC036819790987
:100980008A099B09693271058105910538F0E12FCB
:10099000F0E0E355FB4F80858C2B8087C69511F4E2
:1009A0001F5FC0E8D15051F690E080E0B1CF8F9248
:1009B0009F92AF92BF92CF92DF92EF92FF920F93EE
:1009C0001F93CF93DF938AE0A82EB12CD0E0C0E034
:1009D000EE24EA9493E0F92E88248A9423E0922E60
:1009E000D12CC12C10E000E08FE00E94E103081739
:1009F000190790F1C816D90608F46C0188159905F5
:100A000068F18E159F0508F47C01C80FD91F65E0B9
:100A100070E080E090E00E94210481E0A81AB10813
:100A200019F70C0D1D1DCE01801B910B8E199F090E
:100A30008819990966E070E00E948030CB01DF914F
:100A4000CF911F910F91FF90EF90DF90CF90BF90CB
:100A5000AF909F908F9008958C01D0CF4C01D5CF4F
:100A60002FB7F8946091B3027091B4028091B502EF
:100A70009091B6022FBF0895DC0180E0615090F0A4
:100A80009D919827E92FEF70F0E0E555FD4F2491F7
:100A9000E92FE295EF70F0E0E554FD4FE491822FED
:100AA0008E27ECCF0895DC012C911196ED91FC91ED
:100AB000F8948181822B81839281322F3095932308
:100AC000928387E090E00197F1F78181832381830E
:100AD00083E290E00197F1F790817894EFECF0E0F9
:100AE0003197F1F7922381E009F480E00895FC0149
:100AF00090810180F281E02D292F209560FF14C0A4
:100B0000F8948281822382838181892B8183A3E26D
:100B1000B0E01197F1F78281982B9283789487ED5A
:100B200090E00197F1F70895F894828182238283FF
:100B30008181892B8183AFEFB0E01197F1F782813A
:100B4000982B928378948FE090E0EBCFDF92EF9236
:100B5000FF920F931F93CF93DF93EC01D62EE42ED9
:100B600008E010E0FF24F39461E08D2D8F2109F45B
:100B700060E0CE010E947705FF0C01501109A1F73A
:100B8000E11010C0F894E981FA8191818881809503
:100B900089238183E981FA819281888180958923E3
:100BA00082837894DF91CF911F910F91FF90EF9006
:100BB000DF900895EF92FF920F931F93CF93DF93EF
:100BC0008C017B0140E065E50E94A605E70188E015
:100BD000E80EF11C699140E0C8010E94A605CE15FF
:100BE000DF05C1F7DF91CF911F910F91FF90EF903B
:100BF0000895FC0190810180F281E02DF8948181BB
:100C0000292F20958223818378943DE743E050E0AB
:100C1000315029F1DA011197F1F780818923C1F36D
:100C2000F8948281822382838181892B81837894C5
:100C3000ABE7B7E01197F1F7F894818182238183C4
:100C4000A3E1B1E01197F1F78081982381E009F0E9
:100C500080E07894E3E6F6E03197F1F7089580E0DC
:100C600008956F927F928F929F92AF92BF92CF9290
:100C7000DF92EF92FF920F931F93CF93DF93EC01DC
:100C80007B018A018E819F810E94F905811102C03A
:100C900090E037C0B7018E819F810E94DA0540E065
:100CA0006EEB8E819F810E94A6057801680189E024
:100CB000C80ED11CAE80BF8088E0882E912C712C8C
:100CC00066246394C5010E94530581117628660C41
:100CD000E1E08E1A9108B1F7F70171927F01EC15EE
:100CE000FD0541F78E819F810E94F905813081F6D3
:100CF00068E0C8010E943C0591E0F80120852813B6
:100D0000C7CF892FDF91CF911F910F91FF90EF9067
:100D1000DF90CF90BF90AF909F908F907F906F901B
:100D20000895CF93DF93CDB7DEB729970FB6F89428
:100D3000DEBF0FBECDBFAE014F5F5F4F0E943106D9
:100D4000882331F08D818F33A9F020F48F31A1F009
:100D500080E007C08F3521F08F37D1F78CE001C0DC
:100D60008BE029960FB6F894DEBF0FBECDBFDF91A2
:100D7000CF9108958AE0F5CF89E0F3CF2091CD029D
:100D80003091CE022817390771F49091CB028091EF
:100D9000CC02981741F0E091CB02F0E0EE58FD4F05
:100DA000808190E008958FEF9FEF08950895EF926E
:100DB000FF920F931F93CF93DF93DC015C96ED902E
:100DC000FC905D97E114F10479F481E090E01396D2
:100DD0009C938E93129790E080E0DF91CF911F91CA
:100DE0000F91FF90EF9008955196ED91FC915297DD
:100DF00050968C915097982F90950FB75E962C91A6
:100E00005E97122F127021FD6095F89420811123B6
:100E100019F1282B2083E7012197F1F728E0462FCD
:100E200050E0308160FF1AC0382B3083E7012197F2
:100E3000F1F7BA0175956795215089F7112381F073
:100E40008081892380830FBF5C968D919C9101974F
:100E5000F1F781E090E0C1CF2923DCCF3923E5CF42
:100E60009081892BEFCF2091CD023091CE022817AF
:100E7000390771F48091CC022091CB0290E0805C24
:100E80009F4F821B910960E470E00E9494300895A6
:100E900090E080E008952091CD023091CE02281795
:100EA0003907B9F49091CB028091CC02981789F060
:100EB000E091CB02F0E0EE58FD4F80812091CB0213
:100EC00030E02F5F3F4F2F7333272093CB0290E00A
:100ED00008958FEF9FEF08950F931F930E943005A1
:100EE0006093960470939704809398049093990468
:100EF0008EE894E00E944B0797FF1DC00E943005CA
:100F000000919604109197042091980430919904CF
:100F1000601B710B820B930B009192041091930450
:100F2000209194043091950460177107820793070C
:100F3000F8F28FEF9FEF1F910F910895E091CD028E
:100F4000F091CE02E817F90769F4A389B4899C915E
:100F50008589809589238C931092CE021092CD02C0
:100F600081E0089580E008951092A9041092A804E9
:100F70001092A7041092A6041092A5041092A40443
:100F80008DE991E09093AB048093AA0490919A0428
:100F9000963108F046C02DEB30E03093A504209345
:100FA000A4042BE931E03093A7042093A6042CE29B
:100FB00031E03093A9042093A8042091680084E0D4
:100FC000983048F031E09E3008F430E081E001C014
:100FD000880F3A95EAF7822B809368002DE630E07F
:100FE000983050F02BE630E09E3030F02CE630E0C8
:100FF000963110F030E020E03093A2042093A10459
:10100000292F30E09830C0F581E001C0880F9A9513
:10101000EAF78093A3048091AA049091AB0401970E
:10102000F1F78091A8049091A904892B21F1809176
:10103000CD029091CE0224E08E389207E1F0009725
:1010400011F00E949E078091AC048E7F8093AC04C7
:101050001092CC021092CB028EE894E09093CE02D4
:101060008093CD02E091A104F091A204808190913F
:10107000A304892B808308959E3040F428503109C1
:1010800081E001C0880F2A95EAF7C3CF2E503109BD
:10109000F7CF20914F02260F3327331F213231051E
:1010A000ECF420911703FC0190E080E0243069F01B
:1010B00082E00895A0914F022191AC01415D5D4F06
:1010C000A40FB52FB11D2C930196861798F380912C
:1010D0004F02680F60934F0280E0089581E0089509
:1010E0001092170381E0809316031092F10261E0E1
:1010F00082E10E94820361E083E10E948203E9EBC6
:10110000F0E080818E7F808380818D7F808388E482
:101110008093B80085E48093BC0008951092D002BB
:101120001092CF0210921E03109240030E9470088A
:101130008CE092E09093CA028093C9028DE092E025
:101140009093C8028093C7020895CF93DF9391E0F4
:1011500090932E028823B9F0C091B800D091BA00C4
:101160008091BC008A7B8093BC0060E082E10E9499
:10117000820360E083E10E9482030E947008D093A2
:10118000BA00C093B800DF91CF910895CF92DF925B
:10119000EF92FF920F931F93CF93DF93D091400371
:1011A00081E0D13208F09CC0C0913F030E94FC0353
:1011B0006B017C018091170381116CC082E08093E8
:1011C000170381E0809316038FEF8093150310922D
:1011D0001403D0931303AFE1B3E0E3EFF2E080E058
:1011E000D8138DC01092F2028091F202CC0FC82B5E
:1011F000C093F2028091F102813009F084C0109214
:10120000F1020E94FC036B017C018091F202809349
:10121000BB008091190390911A03A0911B03B09118
:101220001C03892B8A2B8B2BA1F00E94FC030091BD
:10123000190310911A0320911B0330911C036C19A0
:101240007D098E099F09061717072807390708F433
:1012500042C08091BC0083FDD8CF85EC8093BC0058
:101260000E94FC036B017C0180911703823009F41A
:101270004CC0809115038F3F09F469C0809115031C
:10128000803209F466C080911503803309F463C08D
:1012900084E026C08091190390911A03A0911B034A
:1012A000B0911C03892B8A2B8B2B09F483CF0E94CE
:1012B000FC030091190310911A0320911B03309134
:1012C0001C036C197D098E099F090617170728074B
:1012D000390708F06FCF809118030E94A50885E0B8
:1012E00010921E031092400310921D03DF91CF91C4
:1012F0001F910F91FF90EF90DF90CF9008959D91F7
:1013000091938F5F6DCF85EEA9CF80911903909156
:101310001A03A0911B03B0911C03892B8A2B8B2BE2
:1013200009F4A2CF0E94FC030091190310911A0343
:1013300020911B0330911C036C197D098E099F09B4
:10134000061717072807390708F08ECFC4CF80E0AB
:10135000C7CF82E0C5CF83E0C3CFCF92DF92EF92B9
:10136000FF920F931F93CF93DF93D82FC62F613235
:1013700008F098C00E94FC036B017C018091170368
:1013800081116BC081E080931703809316039FEF58
:1013900090931503109214039C0F90931303809362
:1013A000F2028091F202DD0FD82BD093F2028091ED
:1013B000F102813009F078C01092F1020E94FC0322
:1013C0006B017C018091F2028093BB008091190334
:1013D00090911A03A0911B03B0911C03892B8A2BB7
:1013E0008B2BA1F00E94FC030091190310911A03AA
:1013F00020911B0330911C036C197D098E099F09F4
:10140000061717072807390708F448C08091BC0061
:1014100083FDD8CF85EC8093BC000E94FC036B0158
:101420007C0180911703813009F440C0809114033E
:101430008C1710F4C0911403E3EFF2E0A1EDB2E0D9
:1014400080E08C1355C08C2FDF91CF911F910F91AD
:10145000FF90EF90DF90CF900895809119039091C5
:101460001A03A0911B03B0911C03892B8A2B8B2B91
:1014700009F484CF0E94FC030091190310911A0310
:1014800020911B0330911C036C197D098E099F0963
:10149000061717072807390708F070CF809118033F
:1014A0000E94A508C0E0CFCF85EEB5CF809119038B
:1014B00090911A03A0911B03B0911C03892B8A2BD6
:1014C0008B2B09F4AECF0E94FC03009119031091FD
:1014D0001A0320911B0330911C036C197D098E099E
:1014E0009F09061717072807390708F09ACFD6CFA4
:1014F00091919D938F5FA5CFE091D0028091CF0213
:10150000E81730F4F0E0EF52FD4F808190E008954D
:101510008FEF9FEF08959091D0028091CF022FEF2F
:101520003FEF981748F4E92FF0E0EF52FD4F20818C
:1015300030E09F5F9093D002C90108958091CF025F
:101540009091D002891B990B0895CF92DF92EF9270
:10155000FF920F931F93CF93DF937C01CB018A01FE
:1015600020911D03222389F0EB016B01C40ED51ECF
:10157000CC15DD0569F06991D701ED91FC910190E1
:10158000F081E02DC7010995F3CF642F0E9449082F
:10159000C801DF91CF911F910F91FF90EF90DF90E5
:1015A000CF900895CF93DF931F92CDB7DEB76983B5
:1015B00020911D032223F9F020914003203258F09E
:1015C00021E030E0FC013383228390E080E00F9043
:1015D000DF91CF91089580911E03E82FF0E0E15E46
:1015E000FC4F998190838F5F80931E03809340030B
:1015F00081E090E0ECCF61E0CE0101960E944908C5
:10160000F7CF90E080E008958EE894E00E949E0776
:101610000C94B4072F923F924F925F926F927F92F9
:101620008F929F92AF92BF92CF92DF92EF92FF92F2
:101630000F931F93CF93DF93CDB7DEB72D970FB6E0
:10164000F894DEBF0FBECDBF1C010E94040B64E600
:1016500070E080E090E00E9421046AE070E080E0A9
:1016600090E00E942104C101880F991F9D878C87FB
:10167000D12CC12CF12CE12C412C512C320149E010
:1016800050E06AE171E08EE894E00E940F0265E0AC
:1016900070E080E090E00E94210410E000E0812CE6
:1016A000912C54018EE894E00E943307892B39F481
:1016B000F4E08F169104A104B1040CF05FC0023075
:1016C00011050CF05BC08EE894E00E943307892B73
:1016D00099F08EE894E00E944B07E1E0F0E0EC0F17
:1016E000FD1FE00FF11F80836AE070E080E090E072
:1016F0000E9421040F5F1F4F65E070E080E090E0E2
:101700000E9421040230110509F070C089818F3FC9
:1017100009F06CC08A81863809F068C0FE013396F2
:10172000FB87EA878EE894E00E943307892B39F41F
:10173000F4E08F169104A104B1040CF050C00930FC
:10174000110509F059C08B8190E0982F88272C81D2
:10175000820F911D092E000CAA0BBB0B480E591EBF
:101760006A1E7B1E40C0EC85FD85EC15FD0509F069
:1017700086CFE114F10441F4710106C08FEFC81A5D
:10178000D80AE214F3047CF3C301B2010E94C72B10
:101790004B015C01B701FF0C880B990B0E94C72B12
:1017A0009B01AC01C501B4010E94E52D2D960FB639
:1017B000F894DEBF0FBECDBFDF91CF911F910F9187
:1017C000FF90EF90DF90CF90BF90AF909F908F9061
:1017D0007F906F905F904F903F902F9008950430CE
:1017E00011050CF0B0CFFFEFEF1AFF0A8FEF881A48
:1017F000980AA80AB80A56CF8EE894E00E944B07D0
:10180000EA85FB858193FB87EA870F5F1F4F8ACFAD
:10181000FC0124813581232B11F00C943C020895A6
:101820008F929F92AF92BF92CF92DF92EF92FF92F0
:10183000CF93DF93C0E6D4E0988121E020931D038D
:1018400090933F0310921E0310924003682F8EED79
:1018500093E00E94D20A0E94C60863E088810E9439
:10186000AD091092D0028093CF028EED93E00E94DA
:101870008B0A092E000CAA0BBB0B8824982EA92ECC
:10188000BA2E8EED93E00E948B0A092E000CAA0B53
:10189000BB0B6C017D01C828D928EA28FB28FE2C47
:1018A000ED2CDC2CCC248EED93E00E948B0ABC0145
:1018B000990F880B990B6C297D298E299F29DF911F
:1018C000CF91FF90EF90DF90CF90BF90AF909F901F
:1018D0008F9008958F929F92AF92BF92CF92DF9296
:1018E000EF92FF920F931F93209169042F3F19F4F9
:1018F0008AEF0E94100C00916D0410916E0430E08C
:1019000020E0C72ED82EE92EFF24E7FCFA94C01A57
:10191000D10AE20AF30A57E095958795779567957E
:101920005A95D1F7000F111F221F331F4B015C0185
:10193000801A910AA20AB30AA5019401A0916F042A
:10194000B09170040E94082D4B015C01FBE0B5943E
:10195000A79497948794FA95D1F7A7019601C701A8
:10196000B6010E9470309B01AC01ACE055954795E3
:1019700037952795AA95D1F7A0917104B09172047B
:101980000E94082D9B01AC01BEE055954795379507
:101990002795BA95D1F7280D391D4A1D5B1D209357
:1019A0006504309366044093670450936804A5E08F
:1019B000B0E00E94FD2C60587F4F8F4F9F4F672FE4
:1019C000782F892F992787FD9A950E94C72B20E0B1
:1019D00030E048EC52E40E94E52D1F910F91FF90FA
:1019E000EF90DF90CF90BF90AF909F908F90089531
:1019F0002F923F924F925F926F927F928F929F921F
:101A0000AF92BF92CF92DF92EF92FF920F931F930C
:101A1000CF93DF93CDB7DEB76B970FB6F894DEBFE9
:101A20000FBECDBF0E946A0C809169048F3F39F4CC
:101A300087EF0E94100C6E8B7F8B888F998F80911F
:101A4000650490916604A0916704B09168046C01EC
:101A50007D01FF0CCC08DC2C76019C01AD016C2DC6
:101A60007C2D8C2D9C2D345F4140510961097109F9
:101A70008109910929873A874B87652E762E872E13
:101A8000982E9B8F5901C42ED52EE62EF72E082FA7
:101A9000192F0E94A830322E232E488B598B6A8B27
:101AA0007B8B8C8B9D8B3091760420917504932FCA
:101AB000990F990B492F592F692F792F892F0E9440
:101AC000A8300CE00E94A03129833C874A8F5D87B3
:101AD0006E877F87582E492E3091780420917704A5
:101AE000932F990F990BA32CB22CC888D988EA8818
:101AF000FB880C891D89492F592F692F792F892F30
:101B00000E94A83008E00E94B931A980BC84CA8C28
:101B1000DD84EE84FF84052D142D0E94D63170588B
:101B20008F4F9F4FE0917304F09174045F01D12CAB
:101B3000C12CE12CF12C8701E983BA82CB82DC82B3
:101B4000ED82FE820F831887C12CD12CE12CF12C61
:101B500000E010E00E94A83001E20E94B9312A8F13
:101B6000532E49835C876D877E878F87492EA0E03F
:101B70000E94E83109F436C130917E0420917D0441
:101B8000932F990F990BA32CB22CC888D988EA8877
:101B9000FB880C891D89492F592F692F792F892F8F
:101BA0000E94A8301901488B598B6A8B7B8B8C8BD8
:101BB0009D8B30917C0420917B04932F990F990B7E
:101BC000A984BA84CB84D62CE72CF82C092D1B8D44
:101BD000492F592F692F792F892F0E94A83001E1B1
:101BE0000E94A0315101C888D988EA88FB880C89F5
:101BF0001D890E94D63159016A017B01382E192FA7
:101C00004E895F89688D798D84E0759567955795C4
:101C100047958A95D1F780E090E0A0E1B0E0841B81
:101C2000950BA60BB70B3C014D01990C6608762C61
:101C300043019C01AD01662D762D862D962D0FE179
:101C40000E94A031722E832E942E5987B62FA72F73
:101C5000F82FE92F30917A0420917904932F990F6E
:101C6000990B492F592F692F792F892F03E20E9451
:101C7000A031032D0E94D63159016A017B018C01EC
:101C8000272D382D492D59856B2F7A2F8F2F9E2F79
:101C90000E94DF31E5E3AE2EFCE0BF2EC12CD12C3B
:101CA000E12CF12C00E010E00E94A830AA8CB52CA9
:101CB000C980DC84ED84FE840F85142D0E940231DE
:101CC0002F873E8749875A876B8779838C879D87C3
:101CD0000DE00E94B931922E832E742E652E562E61
:101CE000472E382E292E3091840420918304932F7F
:101CF000990F990BA92CB82CC72CD62CE52CF42CB9
:101D0000032D122D492F592F692F792F892F0E94CA
:101D1000A8300E94A83009E10E94B931AF84BE8486
:101D2000C984DA84EB84F9800C851D850E94D63144
:101D300019012A013B014C01309182042091810458
:101D4000932F990F990B492F592F692F792F892F8D
:101D50000E94A83003E10E94B93159016A017B0158
:101D60008C019101A201B301C4010E94D63108E0A7
:101D70000E94B93159016A017B01E82F192F309176
:101D8000800420917F04932F990F990B492F592F8D
:101D9000692F792F892F04E00E94A0310E2F0E9415
:101DA000D6310E948D2E20E030E040E85BE30E94B7
:101DB000262C6B960FB6F894DEBF0FBECDBFDF9119
:101DC000CF911F910F91FF90EF90DF90CF90BF9038
:101DD000AF909F908F907F906F905F904F903F90CB
:101DE0002F90089560E070E0CB01E3CFBF92CF92D7
:101DF000DF92EF92FF920F931F93CF93DF93EC014B
:101E0000B62EC72E8D85811105C0CE010E94F90521
:101E100081110EC01B861D861C8680E0DF91CF914C
:101E20001F910F91FF90EF90DF90CF90BF9008959A
:101E300040E060EFCE010E94A60501E0E12CD12C2C
:101E400011E0CE010E945305F82ECE010E945305E9
:101E500091E0F91218C0813099F51134D8F2DB867F
:101E6000D11002C081E08D878B81882399F223965F
:101E7000EB2DFC2DCF01089629912193E817F90746
:101E8000D9F781E0CBCFEE2DF0E0F8120FC08B85B3
:101E90001817A0F4DE01AE0FBF1F13968C9180239C
:101EA00079F4F12C193008F41C87D12EEC0FFD1FAA
:101EB0008381902F9095892383830AC08113F1CF6A
:101EC000FE01EE0DF11D8381802B8383FF24F394AB
:101ED0006F2DCE010E9477051F5F000F11F4E39470
:101EE00001E087E08E1508F0ACCFB7CFDF92EF921C
:101EF000FF920F931F93CF93DF937C018B01D42E1E
:101F0000DC011696ED91FC911386158614861286D7
:101F10001186108617821682158214821382C0E001
:101F2000B801F701868197810E94F60ED82F882389
:101F300029F0DC1629F0CF5FDC1690F7D0E009C05D
:101F400067E0C8010E943C05D80117969C9189134F
:101F5000F2CF8D2FDF91CF911F910F91FF90EF90D6
:101F6000DF900895CF93909169049F3F41F5682FCA
:101F70008091600491E090931D0380933F03109241
:101F80001E03109240038EED93E00E94D20A0E943D
:101F9000C60862E0809160040E94AD091092D002F0
:101FA0008093CF028EED93E00E948B0AC82F8EEDB6
:101FB00093E00E948B0A20E03C2F282B392B922F94
:101FC000832FCF910895AF92BF92DF92EF92FF924D
:101FD0000F931F93CF93DF935C010AEE13E0D0E0E1
:101FE000C0E0F801D1908F017501EC0EFD1EC70114
:101FF0000E94E72CD81621F06D2DC7010E94EF2C0E
:102000002196CC34D10569F78AEE93E0DF91CF9128
:102010001F910F91FF90EF90DF90BF90AF900895C8
:1020200085ED8093BC008091190390911A03A091D3
:102030001B03B0911C030796A11DB11D23E0B695AB
:10204000A795979587952A95D1F72091BC0024FDF7
:1020500003C01092170308954091190350911A0379
:1020600060911B0370911C03452B462B472B69F392
:102070000097A105B10541F025E32A95F1F700008D
:102080000197A109B109E1CF809118030C94A5082B
:10209000FC0180819181009711F00C94972760E0FA
:1020A00070E0CB010895FB0144815581FC0124813E
:1020B00035812417350778F080819181009759F098
:1020C000FB01608171816115710529F00E94F43373
:1020D00021E0892B09F020E0822F08950F931F93B0
:1020E000CF93DF938C01EB01FC01808191810097FC
:1020F000E1F06881798161157105A9F04281538110
:102100002C813D814217530770F00E94ED338C8182
:102110009D81F801958384831D821C82DF91CF917C
:102120001F910F9108950E94963288819981F8013C
:10213000918380838A819B81938382838C819D811B
:1021400095838483198218821B821A82E5CFCF93EC
:10215000DF93EC0188819981009711F00E949632FB
:10216000198218821D821C821B821A82DF91CF91F4
:102170000895FC0180819181009711F00C949632B2
:1021800008950F931F93CF93DF93EC01888199817A
:10219000009759F02A813B812617370730F081E0FC
:1021A000DF91CF911F910F9108958B016F5F7F4F4A
:1021B0000E941F33009759F0998388831B830A83F9
:1021C0002C813D81232B59F7FC011082E8CF80E060
:1021D000E7CFEF92FF920F931F93CF93DF93611599
:1021E000710541F480E0DF91CF911F910F91FF9035
:1021F000EF90089541155105B1F07B01EC010C8180
:102200001D81040F151FB8010E94C110882351F3CE
:10221000288139818C819D81B701820F931F0E9493
:10222000ED331D830C8381E0DECFFC0144815581B9
:10223000608171818AE594E00C94E910CF93DF937B
:10224000EC01FB0101900020E9F73197AF01461B3B
:10225000570B0E94E910811103C0CE010E94A71004
:10226000CE01DF91CF910895CF93DF93EC01FB0175
:1022700044815581608171810E94E910811103C000
:10228000CE010E94A710CE01DF91CF910895FB01EE
:1022900001900020E9F73197AF01461B570B0C94D2
:1022A000E910EF92FF920F931F93CF93DF93EC010E
:1022B0008B01CB010E94C5277C01BC01CE010E948D
:1022C000C11081110BC0CE010E94A710CE01DF9179
:1022D000CF911F910F91FF90EF900895FD82EC82B6
:1022E000B801888199810E94BE27F0CFFC0111823C
:1022F000108213821282158214820C945111EF9273
:10230000FF920F931F93CF93DF93EC017B018A0120
:10231000BA010E94C11081110BC0CE010E94A7100A
:10232000CE01DF91CF911F910F91FF90EF90089513
:102330001D830C83B701888199810E94ED33F0CF12
:10234000FB0101900020E9F73197AF01461B570BC5
:102350000C947F110F931F93CF93DF93CDB7DEB70C
:1023600062970FB6F894DEBF0FBECDBF8C01CB01D4
:10237000F8011182108213821282158214824AE0BF
:10238000BE016F5F7F4F0E94CE27BE016F5F7F4F00
:10239000C8010E94A01162960FB6F894DEBF0FBE6E
:1023A000CDBFDF91CF911F910F910895CF93DF9310
:1023B000EC01FB018617970749F060817181611577
:1023C000710541F0448155810E947F11CE01DF915A
:1023D000CF9108950E94A710F9CFFC0111821082BD
:1023E00013821282158214820C94D611FC01118280
:1023F00010821382128215821482FB010190002048
:10240000E9F73197AF01461B570B0C947F11CF9220
:10241000DF92EF92FF920F931F93CF93DF936C01A4
:102420007B018A014617570720F48F2D7A01062F6A
:10243000182F6BE571E0C6010E94F611C09152049D
:10244000D0915304EC16FD06F8F40C171D0708F4A0
:10245000E801E0914E04F0914F04EC0FFD1F108154
:10246000108260914E0470914F046E0D7F1DC60165
:102470006115710599F00E94A01180914E04909110
:102480004F04C80FD91F1883C601DF91CF911F9148
:102490000F91FF90EF90DF90CF9008950E94A710CA
:1024A000ECCFEF92FF920F931F93CF93DF93CDB7B3
:1024B000DEB7A1970FB6F894DEBF0FBECDBF7C018B
:1024C000CB01BA01F70111821082138212821582A8
:1024D000148242E0420F8E010F5F1F4F0E9475274A
:1024E000009789F0BC01C7010E94A011A1960FB608
:1024F000F894DEBF0FBECDBFDF91CF911F910F913A
:10250000FF90EF900895C7010E94A710EFCF8F9220
:102510009F92AF92BF92EF92FF920F931F93CF9330
:10252000DF93CDB7DEB72C970FB6F894DEBF0FBEA2
:10253000CDBF64E670E080E090E00E9421048091CD
:102540000401909105010B9731F58091BA0488231D
:1025500009F0F89482E10E9454048C018091BA043D
:10256000882309F078940115110509F4BAC080E0B8
:1025700090ECA9E7B4EC8093AD049093AE04A093E3
:10258000AF04B093B0048093B1049093B204A093CD
:10259000B304B093B404809104019091050146976F
:1025A00031F58091BA04882309F0F89481E00E9403
:1025B00054048C018091BA04882309F078940115A1
:1025C000110509F4EFC080E090ECA9E7B4EC80932A
:1025D000AD049093AE04A093AF04B093B004809385
:1025E000B1049093B204A093B304B093B40464E62E
:1025F00070E080E090E00E942104012B09F060C0AF
:102600004091B1045091B2046091B3047091B4044C
:1026100021E0CE0107960E9451126CE571E0CE01D7
:1026200001960E94F611BE01695F7F4FCE010196AF
:102630000E9434116FE571E00E941E11BC018AE511
:1026400094E00E94D611CE0101960E94B9104091EB
:10265000AD045091AE046091AF047091B00421E0DC
:10266000CE0101960E945112BE016F5F7F4FCE01D5
:1026700007960E946E10CE0101960E94B91063E683
:1026800071E0CE0101960E94F611BE01695F7F4F95
:10269000CE0101960E94341166E671E00E941E117F
:1026A0000E941511CE0101960E94B91064E670E0F7
:1026B00080E090E00E942104CE0107960E94B910AC
:1026C0002C960FB6F894DEBF0FBECDBFDF91CF9131
:1026D0001F910F91FF90EF90BF90AF909F908F90C0
:1026E00008951091B504E090B6046E2D70E090E06E
:1026F00080E00E94C72B2DEC3CEC4CEC5DE30E948B
:10270000262C4B015C01612F70E090E080E00E947C
:10271000C72B9B01AC01C501B4010E94792D6093C8
:10272000AD047093AE048093AF049093B004009115
:10273000B704F090B804602F6F7770E090E080E00D
:102740000E94C72B4B015C016F2D70E090E080E090
:102750000E94C72B2DEC3CEC4CEC5DE30E94262C38
:102760009B01AC01C501B4010E94792D07FD18C081
:102770006093B1047093B2048093B3049093B40453
:102780001E0D100F1F0D81E090E02091B90412136F
:1027900002C090E080E000271127081B190BFBCE38
:1027A0009058E6CF1091B6040091B5046091B5043D
:1027B0007091B60476276727762790E080E00E9424
:1027C000C52B2DEC3CEC4CEC5DE30E94262C609379
:1027D000AD047093AE048093AF049093B004E09086
:1027E000B804F090B7046F2D6F77762F6E2D90E0C0
:1027F00080E00E94C52B2DEC3CEC4CEC5DE30E948C
:10280000262CF7FC18C06093B1047093B204809337
:10281000B3049093B404100F1E0D1F0D81E090E0DF
:102820002091B904121302C090E080E00027112724
:10283000081B190BDCCE9058E6CF4F925F926F9237
:102840007F928F929F92AF92BF92CF92DF92EF9240
:10285000FF92CF93DF93CDB7DEB72C970FB6F894E6
:10286000DEBF0FBECDBF0E94F80C2B013C010E94C1
:102870006A0C4B015C016091F6037091F703809143
:10288000F8039091F9030E94C72B20E030E048EC58
:1028900052E40E94E52D6B017C010E94F80C20E0BF
:1028A00030E048EC52E40E94E52DA70196010E9419
:1028B000E52D21E03EED42E45EE30E94E62E6B0151
:1028C0007C0120E030E048EC52E4C301B2010E94F8
:1028D000E52DAB01BC0122E0CE0101960E94511210
:1028E000BE016F5F7F4F82E494E00E946E10CE01C4
:1028F00001960E94B91062E272E082E494E00E94C4
:10290000471162E474E088E494E00E94D61161E02B
:1029100072E0CE0101960E94F61162E474E0CE01ED
:1029200001960E943411BC0182E494E00E94D61109
:10293000CE0101960E94B9106FE172E08AE594E041
:102940000E94511121E0B501A401CE0101960E941F
:102950005112CE0101960E941511CE0101960E94DE
:10296000B91068E671E08AE594E00E944711A7017A
:10297000960160E070E080E89FE30E94782D20E0FF
:102980003AE24DE257E40E94262CAB01BC0121E063
:10299000CE0101960E945112BE016F5F7F4FCE01A2
:1029A00007960E94ED1164EA71E0CE0107960E943D
:1029B0001E110E941511CE0107960E94B910CE017A
:1029C00001960E94B91062E474E0CE0101960E9463
:1029D000ED116DED71E0CE0101960E941E116AE5C8
:1029E00074E00E943411BC018AE594E00E94D61183
:1029F000CE0101960E94B91065E070E080E090E0A1
:102A00000E9421042C960FB6F894DEBF0FBECDBFF6
:102A1000DF91CF91FF90EF90DF90CF90BF90AF907C
:102A20009F908F907F906F905F904F9008952F921E
:102A30003F924F925F926F927F928F929F92AF924E
:102A4000BF92CF92DF92EF92FF920F931F93CF939B
:102A5000DF93CDB7DEB7CA54D1090FB6F894DEBF05
:102A60000FBECDBF8C016BE571E08AE594E00E945A
:102A7000A011C8010596059740F00C3E2FEF1207F4
:102A800024F01093BE020093BD020C3F4FEF1407D9
:102A900009F4E0C60CF09AC1063F8FEF180709F45D
:102AA000A9C40CF0F4C0043FAFEF1A0784F4013F4F
:102AB000BFEF1B070CF09EC4083E1F4F09F468C708
:102AC0006DE972E08AE594E00E94511193C4043FDD
:102AD000FFEF1F0709F4E7C1053F1F4F89F760E0CB
:102AE00080E10E94B0038091C60281110DC58AE089
:102AF00090E0A0E0B0E02B968CAF9DAFAEAFBFAF43
:102B00002B9765E372E08AE594E00E945111312C25
:102B1000212C26961FAE269727961FAE2797C12CED
:102B2000D12C760102E310E0812C912C540180E13C
:102B30000E94E103092E000CAA0BBB0B880E991E04
:102B4000AA1EBB1E65E070E080E090E00E942104B8
:102B50000150110961F740901204509013046090E5
:102B6000140470901504C501B4010E94C72B20E025
:102B700030E040EA50E40E94262C20E030E040E8BB
:102B80005AE30E94262C20E030E048E452E40E9400
:102B9000E52DA30192010E94782D20E030E040E76E
:102BA00051E40E94262C4B015C01A30192016AE9C9
:102BB00079E989E390E40E94782D9B01AC01C5017D
:102BC000B4010E94E52D20E030E0A9010E94792D9A
:102BD00020E030E040E251E40E94262C5B018C01B1
:102BE000232D322D26964FAD269727965FAD27973A
:102BF0000E94E12E181644F43A2C2B2C26960FAF87
:102C0000269727961FAF27979FEFC91AD90AE90A77
:102C1000F90A2B968CAD9DADAEADBFAD2B978C1543
:102C20009D05AE05BF050CF07DCF6EE170E080E044
:102C300090E00E94210422E0432D522D26966FAD94
:102C4000269727967FAD2797CE0180960E94511236
:102C500069E971E0CE0101960E94F611BE01605E45
:102C60007F4FCE0101960E9434116AE574E00E9404
:102C70003411BC018AE594E00E94D611CE01019680
:102C80000E94B910CE0180960E94B910B3C30B3FC9
:102C90004FEF14070CF0CFC5093F5FEF15070CF09D
:102CA000A9C3073F8FEF180709F433C4083F1F4F2C
:102CB00009F006CF0E9430052B013C018EE894E01C
:102CC0000E949E0764E670E080E090E00E9421048C
:102CD0000E94B40764E670E080E090E00E94210466
:102CE00026961FAE2697B12CA12CD12CC12CF12CED
:102CF000E12C1E01B0E22B0E311C0E94300564193C
:102D0000750986099709683B7B408105910508F0A4
:102D1000D8C48EE894E00E943307892B09F44FC091
:102D20008CED95E0A0E0B0E0809392049093930442
:102D3000A0939404B09395040E946C0797FD3FC044
:102D400082349105C9F78E010F5F1F4F48010E9421
:102D50006C0797FFAEC489818D3489F5C8014D9603
:102D600030E020E0F80141918F01240F311DE81778
:102D7000F907C1F72E5B3F4F8E8D90E0982F882783
:102D80004F8D840F911D28173907C9F4EC80F12C61
:102D9000FE2CEE248D81E80EF11CCE80D12CDC2C93
:102DA000CC248F81C80ED11CA884B12CBA2CAA24A3
:102DB0008985A80EB11CF1E02696FFAF269762E345
:102DC00070E080E090E00E94210497CF033011056D
:102DD00009F443C544F510161106ACF00F3FAFEFF0
:102DE0001A070CF007C30D3F1F4F09F069CE81E0B1
:102DF0008093C6028091BD029091BE029093C10261
:102E00008093C002F7C20130110509F449C00230B5
:102E1000110509F055CE80910101882309F4EAC219
:102E20000E941D14E7C20A301105B4F406301105E2
:102E30000CF0E0C20430110509F48FC5053011050E
:102E400009F03ECE62E972E08AE594E00E945111F9
:102E50000E94D704BC0191C50138110509F030CE9C
:102E6000809101018823B1F00E941D146AE574E08D
:102E7000CE0101960E94ED11CE0101960E94080C30
:102E8000CE0101960E94B91064EF71E080E090E0FD
:102E90000E94210464EF71E080E090E00E94210430
:102EA0000E948712A7C260E08FE00E94B003EAEBA5
:102EB000F3E0E491E8A3E6EAF3E0E491F0E0EE0F5A
:102EC000FF1FED57FC4F859194919AA389A31BA6F0
:102ED0001DA61CA6CE01809698878F831D821E8218
:102EE000198289E08A8381E08B838C831C8A1B8A08
:102EF0001AA619A618A61FA21EA21DA21CA21BA2DA
:102F000001E0BE01625D7F4F8F8198850E94F60EC1
:102F1000882309F45BC067E0CE018E960E943C05D1
:102F20009DA98913EECF898181111DC08F8198855C
:102F30000E94F905BE01625D7F4F8F8198850E94D6
:102F4000DA0540E064EB8F8198850E94A6058F81A9
:102F500098850E945305182F8F8198850E94F90546
:102F6000111101C009831A818EA5803109F414C59D
:102F7000BE01625D7F4FCE0101960E9491068117CE
:102F800090F48A818A838D818F5F8D838EA58832AC
:102F900031F0B0F4803119F0823209F0B2CF8E8175
:102FA0008F5F8E83AECF8EA5803111F48CE0EACF97
:102FB000BE01625D7F4FCE0101960E949106E2CF75
:102FC0008B3369F3823409F09CCFE9CF8F819885E8
:102FD0000E94F90540E06CEC8F8198850E94A6055F
:102FE000498164E48F8198850E94A6058B8188239E
:102FF00079F1EA81E9503EEEC32E32E0D32EE33080
:1030000038F4F0E0EE0FFF1FEC5EFE4FC080D18081
:103010008C81882309F461C0898181115EC00E947E
:1030200030054B015C010D2C000CEE08FF088F8170
:1030300098850E945305813059F00E9430056C1923
:103040007D098E099F09681579058A059B0578F326
:103050008CE08A83F12CE12C0FE58FE7D82E9FE1DD
:10306000C92E2FE3B22E8D818E151F0409F00CF4AA
:1030700099C04E2DBE01695C7F4FCE0101960E9422
:10308000760F1A811D3080F11CE08FA9803181F10B
:10309000BE01695C7F4FCE0101960E9491068117A7
:1030A00009F478C0AE01425D5F4FBE01695C7F4F9D
:1030B000CE0101960E943106882309F46BC08FA9C6
:1030C000803109F467C01B3009F468C01C3091F0EE
:1030D0001A3009F065C0BAAA0EC0B601DD0C880B23
:1030E000990B0E942104B4CF193078F619E0CDCFA6
:1030F0008CE0D5CFDAAA8F8198850E94F905BE01B0
:10310000695C7F4F8F8198850E94DA0540E06EE40C
:103110008F8198850E94A60540E068A98F819885D7
:103120000E94A60540E069A98F8198850E94A605A6
:103130008FA9803131F040E06AA98F8198850E9483
:10314000A6058F8198850E94F905BE01695C7F4FB5
:103150008F8198850E94DA05498168E48F8198857E
:103160000E94A60564E170E080E090E00E942104E6
:103170008981882331F06AE070E080E090E00E946D
:1031800021048F8198850E94F9058A81811708F4AE
:10319000812F8A83EFEFEE1AFE0A65CF0AABABCF21
:1031A000CAAAA9CFEE80F12C62E272E0E114F10428
:1031B00009F488CC6BE571E08AE594E00E94A011E7
:1031C0006701F5E0EF16F1041CF014E0C12ED12CDC
:1031D000B6E1AB2EB4E0BB2E10E000E0402FBE0104
:1031E000695C7F4FCE0101960E94760F811139C034
:1031F00020E030E04EEF52ECF50161917191819148
:1032000091915F010E94792D2B013C010F5F1F4FAF
:1032100020E030E04CEF52EC0E94C02B87FF6DC0E5
:10322000B801CE01C7960E94AA116EE671E0CE01E8
:103230008E960E94F611BE01695C7F4FCE018E967C
:103240000E94341160E771E00E941E110E94151166
:10325000CE018E960E94B910CE01C7960E94B91079
:1032600096C0AE01425D5F4FBE01695C7F4FCE01EB
:1032700001960E943106882309F4BACF6FA570E049
:10328000762F6627770F770F770F2EA548E0249FBC
:1032900090011124262B372B8FA98031D1F46DA9F1
:1032A00070E08CA9DB01A81BB109CD019695982F80
:1032B0008827979587950E949430CB014097B90154
:1032C000F3E0660F771FFA95E1F760789C01260F0F
:1032D000371F2138B4EE3B070CF48ACFB901330F06
:1032E000880B990B0E94C72B20E030E040E05CE3A4
:1032F0000E94262C9B01AC017FCF22E0B301A201EA
:10330000CE01F3E0EF16F10409F4A8C0CF960E94B5
:103310005112B801CE01C7960E94AA116EE671E063
:10332000CE018E960E94F611BE01695C7F4FCE01E0
:103330008E960E94341166EB71E00E941E11BE0150
:10334000615C7F4F0E943411BC0182E494E00E94D2
:10335000D611CE018E960E94B910CE01C7960E945A
:10336000B910CE01CF960E94B91062E474E0CE018C
:103370008E960E94ED116DED71E0CE018E960E9449
:103380001E110E941511CE018E960E94B9100C15C7
:103390001D050CF423CFA0905A04B0905B04A11437
:1033A000B10449F000915E0410915F0465010115BC
:1033B000110509F06DC0F3E0EF16F104A9F46CE714
:1033C00071E0CE018E960E94F6116AE574E0CE019E
:1033D0008E960E943411BC018AE594E00E94D611B9
:1033E000CE018E960E94B91066E871E08AE594E0FD
:1033F0000E94471180915E0490915F04892B71F0C7
:103400006AE574E0CE0101960E94ED11CE010196AD
:103410000E94080CCE0101960E94B91064E670E08B
:1034200080E090E00E942104C65BDF4F0FB6F89465
:10343000DEBF0FBECDBFDF91CF911F910F91FF90E7
:10344000EF90DF90CF90BF90AF909F908F907F9044
:103450006F905F904F903F902F9008958E960E94AE
:103460005112BE01625D7F4FCE01C7960E94ED11E1
:103470006DED71E0CE01C7960E941E110E941511DC
:10348000CE01C7960E94B910CE018E96E7CE640198
:1034900046012FEF821A920AD6018C91082E000C59
:1034A000990B0E948F2B892B91F7015011090A0D5E
:1034B0001B1DF8018081082E000C990B0E948F2B98
:1034C000892B31F00C151D0518F001501109F1CFB1
:1034D000A8014F5F5F4F4C195D0950935F04409303
:1034E0005E04AC14BD0420F4B601C5010E94E433AF
:1034F000E0915A04F0915B0480915E0490915F0426
:10350000E80FF91F108257CF83E090E0A0E0B0E011
:10351000F2CA68EC70E080E090E00E9421040E9412
:10352000040B64E670E080E090E00E94210462E316
:1035300070E080E090E00E94210449E050E06AE100
:1035400071E08EE894E00E940F0262E370E080E098
:1035500090E00E94210403E010E08EE894E00E94D5
:103560003307892B61F149E050E06AE171E08EE8B0
:1035700094E00E940F0265E070E080E090E00E941D
:103580002104F12CE12C8EE894E00E94330792E0B4
:10359000E916F104A4F48EE894E00E943307892B25
:1035A00039F08EE894E00E944B07AFEFEA1AFA0A6E
:1035B00065E070E080E090E00E942104E4CF62E3E7
:1035C00070E080E090E00E9421040150110929F68A
:1035D0008AE090E00E940A0B6B017C0120E030E061
:1035E000A9010E94C02B181634F08AE090E00E94D6
:1035F0000A0B6B017C010BE010E020E030E042EDB3
:1036000053E4C701B6010E94C02B181684F0015084
:10361000110969F068EC70E080E090E00E942104FC
:1036200083E090E00E940A0B6B017C01E6CF20E072
:1036300030E0A901C701B6010E94C02B69E472E025
:1036400018160CF03FCA20E030E048EC52E4C70105
:10365000B6010E94C02B21E087FF20E0B701A60140
:10366000CE0101960E945112BE016F5F7F4F8AE525
:1036700094E00E946E10CE0101960E94B9106DE98F
:1036800071E0CE0101960E94F6116AE574E0CE0168
:1036900001960E94341162EA71E00E941E11BC0181
:1036A0008AE594E00E94D611CE0101960E94B910DD
:1036B000A1CED4018D934D01A215B30509F047CBDE
:1036C0004ACB0E9430056419750986099709683B41
:1036D0007B4081059105A8F426964FAD269744239B
:1036E00009F49CC062E370E080E090E00E94210455
:1036F0008EE894E00E949E0762E370E080E090E034
:10370000A6C026965FAD2697552309F487C0B5015C
:10371000CE0180960E94AA11B601CE018E960E941B
:10372000AA11B701CE01CF960E94AA11BE01615C19
:103730007F4FCE01C7960E94ED1166EA71E0CE017F
:10374000C7960E941E11BE01625D7F4F0E94341118
:1037500066EA71E00E941E11BE01605E7F4F0E940A
:103760003411BC018AE594E00E94D611CE01C796BF
:103770000E94B910CE01CF960E94B910CE018E964C
:103780000E94B910CE0180960E94B910B501CE01F9
:1037900080960E94AA11B601CE018E960E94AA11AF
:1037A000B701CE01C7960E94AA1168EA71E0CE0166
:1037B000CF960E94F611BE01695C7F4FCE01CF9675
:1037C0000E9434116DED71E00E941E11BE01625D18
:1037D0007F4F0E9434116DED71E00E941E11BE01F9
:1037E000605E7F4F0E94341168EB71E00E941E11F1
:1037F000BC018AE594E00E94D611CE01CF960E94CA
:10380000B910CE01C7960E94B910CE018E960E94C3
:10381000B910CE0180960E94B91064CF67E672E0BD
:103820008AE594E00E94511168E572E08AE594E02F
:103830000E94511157CF8091C602882321F08AE55A
:1038400094E00E943C0268EC70E080E090E00E940E
:103850002104D0CD1092C602CDCD62E772E08AE598
:1038600094E00E9451118BE0E82EF12C10E000E072
:103870009924939493E2892E90921D0380923F03A2
:1038800010921E031092400362E083E20E94AD0991
:103890001092D0028093CF028EED93E00E948B0AAB
:1038A000D82EC12C8EED93E00E948B0A5C01AC28CF
:1038B000BD280E94C608B50190E080E00E94C52B9B
:1038C0002AE939E949E95FE30E94E52D0E945E2E6D
:1038D0000617170708F48B0162E370E080E090E0C0
:1038E0000E94210481E0E81AF10831F619A218A219
:1038F0001BA21AA21DA21CA24AE0BE016F5F7F4F4D
:10390000C8010E94EE27BE016F5F7F4FCE018096F7
:103910000E94A0116EEB71E0CE0101960E94F6119B
:10392000BE01605E7F4FCE0101960E94341161ECB2
:1039300071E00E941E116AE574E00E943411BC011E
:103940008AE594E00E94D611CE0101960E94B9103A
:10395000CE0180960E94B910CFCE81E08093000105
:103960000E94D7048C0162E872E08AE594E00E942C
:10397000511160E074E0601B710BCE0101960E9452
:10398000AA11CE0101960E941511CE0101967CC9A3
:10399000F0E0E0E009952ECD1D3008F0F2CA06CB2C
:1039A0001F920F920FB60F9211242F933F934F93B4
:1039B0005F936F937F938F939F93AF93BF93EF9397
:1039C000FF9381E493E00E94A602FF91EF91BF91E3
:1039D000AF919F918F917F916F915F914F913F91A7
:1039E0002F910F900FBE0F901F9018951F920F925E
:1039F0000FB60F9211242F938F939F93EF93FF9302
:103A0000E0915103F09152038081E0915703F091CE
:103A1000580382FD1BC0908180915A038F5F8F7382
:103A200020915B03821741F0E0915A03F0E0EF5BD5
:103A3000FC4F958F80935A03FF91EF919F918F9147
:103A40002F910F900FBE0F901F9018958081F4CF8B
:103A50001F920F920FB60F9211242F933F938F93C3
:103A60009F93AF93BF938091B3029091B402A091C2
:103A7000B502B091B6023091B20223E0230F2D3788
:103A800058F50196A11DB11D2093B2028093B30297
:103A90009093B402A093B502B093B6028091B7029E
:103AA0009091B802A091B902B091BA020196A11DFD
:103AB000B11D8093B7029093B802A093B902B0935E
:103AC000BA02BF91AF919F918F913F912F910F902B
:103AD0000FBE0F901F90189526E8230F0296A11D88
:103AE000B11DD2CF1F920F920FB60F9211242F93B8
:103AF0003F934F935F936F937F938F939F93AF9376
:103B0000BF93EF93FF93E091CD02F091CE023097F7
:103B100049F0A685B7858585968D91FF14C09C9147
:103B20008923A1F4FF91EF91BF91AF919F918F9164
:103B30007F916F915F914F913F912F910F900FBEA9
:103B40000F901F9018959C91892361F7A389B489E0
:103B50009C918589809589238C9386899789019783
:103B6000F1F7608D718DA685B785558538E020E029
:103B7000CB010197F1F7822F90E095958795282F3B
:103B80004C91452309F02068315091F7868D81FDD5
:103B900020958091CC0290E001968F739927309107
:103BA000CB02381799F0A091CC02B0E0AE58BD4FCF
:103BB0002C938093CC02828D938D0197F1F7A3898A
:103BC000B4898C919589892B8C93ACCF868D81603B
:103BD000868FF1CF1F920F920FB60F9211242F9361
:103BE0003F934F935F936F937F938F939F93AF9385
:103BF000BF93EF93FF938091B900887F803609F4DB
:103C00004AC0F0F5883209F4A7C018F5803109F4EC
:103C10009BC0B8F4882309F4F9C0883009F494C033
:103C2000FF91EF91BF91AF919F918F917F916F9194
:103C30005F914F913F912F910F900FBE0F901F906A
:103C40001895883109F488C0803251F780931503A4
:103C500014C0803409F49DC040F48033B9F3883334
:103C6000F9F68093150385ECB0C0803509F485C062
:103C7000883509F496C0883499F60E941010D0CF88
:103C8000883909F48CC038F5883729F050F4883623
:103C900011F0803729F683E08093170310927102A8
:103CA00057C0883809F47BC0803919F0803809F092
:103CB000B7CF80917102803208F071C0E09171023B
:103CC00081E08E0F809371028091BB00F0E0EF5A8B
:103CD000FD4F80833DC0803B39F0E0F4803A09F429
:103CE00079C0883A09F09CCF84E080931703109242
:103CF000500210924F02E091C902F091CA02099558
:103D000080914F0281110FC081E080934F02109289
:103D10002F0209C0803C09F4A6CF883C09F4A3CF48
:103D2000883B09F07DCFE091500281E08E0F8093B7
:103D30005002F0E0E15DFD4F80818093BB009091E7
:103D4000500280914F0229C08091F2028093BB0003
:103D500085EC8093BC0064CF909114038091130391
:103D6000981758F5E091140381E08E0F80931403A7
:103D7000F0E0ED50FD4F8081E9CFE091140381E048
:103D80008E0F809314038091BB00F0E0ED50FD4F47
:103D9000808390911403809113039817C8F285E8EB
:103DA000D8CFE091140381E08E0F809314038091AB
:103DB000BB00F0E0ED50FD4F808380911603811130
:103DC0005CCF81E08093F10284EA8093BC00109282
:103DD000170326CF85EC8093BC00109217038091C7
:103DE0007102803230F4E0917102F0E0EF5AFD4F41
:103DF00010826091710270E0E091C702F091C802F8
:103E000081E592E00995109271020ACF1092150394
:103E100034CF109244031092430388EE93E0A0E065
:103E2000B0E08093450390934603A0934703B0937B
:103E3000480327E231E0309342032093410325EC0D
:103E400030E030934E0320934D0324EC30E0309368
:103E5000500320934F0320EC30E030935203209323
:103E6000510321EC30E0309354032093530322ECB0
:103E700030E0309356032093550326EC30E0309326
:103E800058032093570310925A0310925B03109229
:103E90005C0310925D031092E1031092E0038093A3
:103EA000E2039093E303A093E403B093E50329E3D3
:103EB00031E03093DF032093DE031092BA041092B6
:103EC0009104109290048093920490939304A09391
:103ED0009404B09395048BE491E090938F048093C5
:103EE0008E041092A5041092A4041092A7041092BC
:103EF000A6041092A9041092A8041092AB04109288
:103F0000AA046091AC046E7F6D7F6093AC046695EB
:103F1000617081E0682789E00E94820361E089E0A6
:103F20000E94B003E4EBF3E0E491E0939E04E0EA46
:103F3000F3E0E491F0E0EE0FFF1FE357FC4F8591B3
:103F400094919093A00480939F0460E08AE00E9483
:103F5000B0038091AC0481FD04C061E08AE00E945E
:103F600082038AE080939A04E5EBF3E0E491E09326
:103F70009B04E1EAF3E0E491F0E0EE0FFF1FED5760
:103F8000FC4F8591949190939D0480939C048FEFB6
:103F90008093690480936A0480936B0480936C041B
:103FA0006BE571E08AE594E00E94F6116BE571E043
:103FB00084E594E00E94F6116BE571E08EE494E0F4
:103FC0000E94F6116BE571E088E494E00E94F6111E
:103FD0006BE571E082E494E00E94F61166EC71E01A
:103FE0008CE394E00E94F6116DEC71E086E394E0BE
:103FF0000E94F61186E190E09093EB038093EA0330
:104000008CE79CE8A1E0B0E08093F6039093F7037F
:10401000A093F803B093F90381EA97E6A3E3BDEB1D
:104020008093FA039093FB03A093FC03B093FD03EA
:1040300086E696E6A6EABFE38093FE039093FF032D
:10404000A0930004B093010481E080930A0429E165
:1040500030E030930C0420930B0480930D0480E037
:1040600090E4ACE1B5E480930E0490930F04A09328
:104070001004B093110410921204109213041092C1
:10408000140410921504E6E1F4E080E1DF011D92D2
:104090008A95E9F7109226041092270410922804BA
:1040A0001092290410922A0410922B0410922C04CE
:1040B00010922D0410922E0410922F0410923004AE
:1040C000109231041092320410923304109234048E
:1040D000109235040895CF93DF93CDB7DEB72C97B8
:1040E0000FB6F894DEBF0FBECDBF789484B5826062
:1040F00084BD84B5816084BD85B5826085BD85B58C
:10410000816085BD80916E00816080936E00109209
:104110008100809181008260809381008091810084
:104120008160809381008091800081608093800015
:104130008091B10084608093B1008091B000816073
:104140008093B00080917A00846080937A0080919F
:104150007A00826080937A0080917A0081608093F7
:104160007A0080917A00806880937A001092C10072
:1041700061E08EE00E94B003E0915103F0915203A0
:1041800082E08083E0914D03F0914E031082E09134
:104190004F03F09150038FEC808310925903E0910C
:1041A0005503F091560386E08083E0915303F0912C
:1041B0005403808180618083E0915303F091540324
:1041C000808188608083E0915303F0915403808163
:1041D00080688083E0915303F091540380818F7D48
:1041E000808360E08EE00E9482030E948E0881E05E
:1041F00080931D0383E280933F0310921E0310926D
:10420000400360E18EED93E00E94D20A0E94C6084E
:104210008FE39CE90197F1F700C0000068EC70E0C3
:1042200080E090E00E94210484E690E090930301F6
:10423000809302010E94E72C8093BB0285E690E008
:104240000E94E72C8093BC020091BB021091BC023B
:10425000B801012E000C880B990B0E94C72B9B0103
:10426000AC010E94362F811106C00B5011090C3091
:10427000110508F4A9C084E690E00E94E30F68EC01
:1042800070E080E090E00E94210461EE72E08AE537
:1042900094E00E9451116AE574E0CE0101960E94FB
:1042A000ED11CE0101960E94080CCE0101960E94EC
:1042B000B9100E948E0864E670E080E090E00E94F1
:1042C000210486E780936004809169048F3F11F494
:1042D0000E948E08809169048F3F01F580916004EF
:1042E00091E090931D0380933F0310921E03109260
:1042F000400360ED8EED93E00E94D20A0E94C60852
:1043000061E0809160040E94AD091092D002809318
:10431000CF028EED93E00E948B0AF82EF8E5FF168F
:1043200009F47DC065ED72E08AE594E00E945111C8
:10433000109201016AE574E0CE0101960E94ED1130
:10434000CE0101960E94080CCE0101960E94B91080
:1043500098EE892E93E0992EA12CB12C712C612C12
:104360002AE2E22EF12C80E0C82E80E0D82E6BE508
:1043700071E0CE0107960E94F61110E081E493E00F
:104380000E948602181619060CF0D9C01111D7C068
:1043900081E493E00E9464028A3009F4B1C08D3058
:1043A00009F4AEC089831A8241E050E0BE016F5F1C
:1043B0007F4FCE0107960E94E9106AE070E080E02E
:1043C00090E00E942104DACF3AEEC32E33E0D32EE0
:1043D00004E610E0C8010E94E72CF60181936F010A
:1043E0000F5F1F4F003B1105A9F78091EA039091E1
:1043F000EB0390930501809304016CEE73E0CE0112
:1044000001960E94F611BE016F5F7F4F8CE394E02E
:104410000E946E10CE0101960E94B91030CF88E83C
:104420000E94B20F90936E0480936D048AE80E94FC
:10443000B20F9093700480936F048CE80E94B20FC7
:1044400090937204809371048EE80E94B20F90934F
:1044500074048093730480E90E94B20F90937604F1
:104460008093750482E90E94B20F90937804809340
:10447000770484E90E94B20F90937A0480937904C0
:1044800086E90E94B20F90937C0480937B0488E9B4
:104490000E94B20F90937E0480937D048AE90E946B
:1044A000B20F9093800480937F048CE90E94B20F36
:1044B00090938204809381048EE90E94B20F9093BE
:1044C000840480938304809169048F3F09F040CF76
:1044D0008091600491E090931D0380933F031092BC
:1044E0001E031092400364EF8EED93E00E94D20A07
:1044F0006FE38EED93E00E94D20A0E94C60828CF97
:104500001091BF021123C9F08B859C85892B09F47A
:1045100054CF66ED71E0CE0101960E94F611BE0106
:10452000695F7F4FCE0101960E9434110E943C02C8
:10453000CE0101960E94B91040CF11E03ECFBE01DE
:10454000695F7F4F8EE494E00E946E10CE01079663
:104550000E94B9106BE571E08AE594E00E94A01119
:1045600080915204909153048130910509F0AFC0BD
:104570006EE474E0CE0101960E94ED118D819E8162
:10458000892B89F0E981FA81309769F08081823442
:10459000A9F1BCF48A3209F497C0813441F168EE84
:1045A00071E0833231F1BE016F5F7F4F8EE494E0A2
:1045B0000E94D6116AE070E080E090E00E94210441
:1045C00029C08136A1F074F4833469F765EE71E097
:1045D0008EE494E00E94A01121E02093C6028DEFAA
:1045E0009FEF16C0823651F0833681F3DCCF6FED3A
:1045F00071E08EE494E00E94A0110CC062EE71E0C4
:104600008EE494E00E94A0111092C6028CEF9FEFFE
:104610000E941715CE0101960E94B9108EE494E015
:104620000E944810CB010E9417158091C602882372
:1046300009F43EC00E943005A50194010E94472D57
:10464000CA01B9010E94C52B2091C2023091C30258
:104650004091C4025091C5020E94782D20910A0118
:1046600030910B0140910C0150910D010E94E12EFF
:104670001816F4F40E943005A50194010E94472DFC
:10468000CA01B9010E94C52B6093C2027093C30294
:104690008093C4029093C5028091C0029091C102A0
:1046A0000E9417156AE070E080E090E00E9421040B
:1046B000C114D10409F45BCE0E949202882309F44C
:1046C00056CE0E9400004FCE6BEE71E092CF049761
:1046D00068F56EEE71E0CE0101960E94F611BE0102
:1046E0006F5F7F4F8EE494E00E945310182FCE012D
:1046F00001960E94B9101123C9F080915204909143
:104700005304029788F0E0914E04F0914F043097E3
:1047100059F0818180330CF4845EF701E81BF109C4
:1047200087FDF395CF017FCF80E0F6CF6EE474E094
:1047300084E594E00E94D611009154041091550430
:104740000115110571F0F80181918F01882349F05D
:10475000082E000C990B0E94DC33F80131978083FE
:10476000F2CF68E673E0CE0101960E947611BE0199
:104770006F5F7F4F84E594E00E945310182FCE01A5
:1047800001960E94B910112319F0F30109954DCF3C
:1047900060E673E0CE0101960E947611BE016F5F64
:1047A0007F4F84E594E00E945310182FCE010196AC
:1047B0000E94B910112399F160EF71E0CE010196CA
:1047C0000E94F61166E374E0CE0101960E94341156
:1047D000BC018AE594E00E94D611CE0101960E94A8
:1047E000B9106AEF71E0CE0101960E94F6116AE5F8
:1047F00074E0CE0101960E943411BC01CE010796EF
:104800000E94ED11CE0107960E94080CCE0107967A
:104810000E94B910CE0101960E94B91006CF69E539
:1048200073E0CE0101960E947611BE016F5F7F4F4B
:1048300084E594E00E945310182FCE0101960E9447
:10484000B910112359F06BE473E08AE594E00E94FB
:1048500051118CE394E00E941511C3CF64E473E01E
:10486000CE0101960E947611BE016F5F7F4F84E5F5
:1048700094E00E945310182FCE0101960E94B910A7
:10488000112301F147E050E066E070E0CE010196AF
:104890000E940712BE016F5F7F4F88E494E00E9480
:1048A0006E10CE0101960E94B91088E494E00E9437
:1048B0004810672B19F41092BF02B7CEF1E0F093C5
:1048C000BF02B3CE6DE373E0CE0101960E94761174
:1048D000BE016F5F7F4F84E594E00E945310182F54
:1048E000CE0101960E94B910112309F479C04091BC
:1048F0005204509153044730510508F496CE66E0B7
:1049000070E0CE0101960E940712BE016F5F7F4FDB
:1049100088E494E00E946E10CE0101960E94B910C6
:104920008091480490914904009709F455C00E9471
:10493000932760930A0170930B0180930C0190936D
:104940000D0162E373E08AE594E00E945111409109
:104950000A0150910B0160910C0170910D0122E050
:10496000CE0101960E945112BE016F5F7F4FCE01B2
:1049700007960E94ED116CEF71E0CE0107960E9440
:104980001E110E941511CE0107960E94B910CE018A
:1049900001960E94B9106AE574E0CE0101960E946A
:1049A000ED11CE0101960E94080CCE0101960E94E5
:1049B000B9100E943005A50194010E94472DCA013B
:1049C000B9010E94C52B6093C2027093C302809309
:1049D000C4029093C50229CE60E070E0CB01A9CF5C
:1049E0006BE273E0CE0101960E947611BE016F5F0B
:1049F0007F4F84E594E00E945310182FCE0101965A
:104A00000E94B910112309F467C0409152045091DB
:104A100053044730510508F408CE66E070E0CE013B
:104A200001960E940712BE016F5F7F4F88E494E0F9
:104A30000E946E10CE0101960E94B9108091480428
:104A400090914904009709F443C00E949327609312
:104A5000060170930701809308019093090160E2B9
:104A600073E08AE594E00E94511140910601509153
:104A70000701609108017091090121E0CE010196C2
:104A80000E945112BE016F5F7F4FCE0107960E94B8
:104A9000ED116CEF71E0CE0107960E941E110E948D
:104AA0001511CE0107960E94B910CE0101960E9401
:104AB000B9106AE574E0CE0101960E94ED11CE01B5
:104AC00001960E94080CCE0101960E94B910ADCD4E
:104AD00060E070E0CB01BBCF6BE173E0CE010196EB
:104AE0000E947611BE016F5F7F4F84E594E00E94C3
:104AF0005310182FCE0101960E94B910112331F1E5
:104B000046E050E064E070E0CE0101960E9407129A
:104B1000BE016F5F7F4F88E494E00E946E10CE016B
:104B200001960E94B91088E494E00E9448107093A6
:104B3000EB036093EA037093050160930401809195
:104B40000201909103010E94E30F6FCD67E173E0D2
:104B5000CE0101960E947611BE016F5F7F4F84E502
:104B600094E00E945310182FCE0101960E94B910B4
:104B7000112309F44FC0409152045091530463E053
:104B800070E0CE0101960E940712BE016F5F7F4F59
:104B900088E494E00E946E10CE0101960E94B91044
:104BA00068E474E0CE0101960E94ED111F82188620
:104BB00041E050E0BE01695F7F4FCE0101960E9447
:104BC000E910811104C0CE0101960E94A710BE0118
:104BD0006F5F7F4F8CE394E00E94D611CE01019667
:104BE0000E94B91000914004109141040115110573
:104BF00009F4A5CF0150110960913C0470913D0466
:104C0000A8018CEE93E00E940234F801E451FC4FBD
:104C1000108295CF64E173E0CE0101960E94761177
:104C2000BE016F5F7F4F84E594E00E945310182F00
:104C3000CE0101960E94B910112309F48AC0409157
:104C40005204509153044031510508F0EECC62E01B
:104C500070E0CE0101960E940712BE016F5F7F4F88
:104C600088E494E00E946E10CE0101960E94B91073
:104C70008091480490914904009799F10E949327EC
:104C800020E030E048EC52E40E94262C0E94572E8F
:104C90006093F6037093F7038093F8039093F903FE
:104CA0008B019C0100591F452140310901341C49E9
:104CB00021053105D0F06EEF71E0CE0101960E9422
:104CC000F61168E474E0CE0101960E94341164E0AC
:104CD00072E00E941E11BC018AE594E00E94D61188
:104CE00099CD60E070E0CB01CBCF0E94C72B20E0D4
:104CF00030E048EC52E40E94E52DAB01BC0122E01B
:104D0000CE0101960E945112BE016F5F7F4F8AE56E
:104D100094E00E946E10CE0101960E94B91064E1E9
:104D200072E0CE0101960E94F6116AE574E0CE01B0
:104D300001960E94341161E272E00E941E11BC01D2
:104D40008AE594E00E94D611CE0101960E94B91026
:104D5000F6CE66E272E0CE0101960E94F611BE0127
:104D60006F5F7F4F84E594E00E945310182FCE01AF
:104D700001960E94B910112309F45EC009E110E008
:104D8000212C312C210180E10E94E103BC01990F0B
:104D9000880B990B0E94C72B9B01AC01C201B1018A
:104DA0000E94792D1B012C016AE070E080E090E008
:104DB0000E9421040150110931F720E030E040EA5F
:104DC00050E4C201B1010E94262C20E030EC4FE7F4
:104DD00054E40E94E52D20E030E048EC51E40E94CC
:104DE000E52D609312047093130480931404909340
:104DF000150480910201909103010E94E30F61E08C
:104E000073E08AE594E00E945111409112045091A0
:104E10001304609114047091150422E0CE010196F0
:104E20000E945112BE016F5F7F4FCE0107960E9414
:104E3000ED116AE272E02FCE6DEF72E0CE010196C5
:104E40000E947611BE016F5F7F4F84E594E00E945F
:104E50005310182FCE0101960E94B910112309F4A6
:104E6000E4CB409152045091530463E070E0CE01D2
:104E700001960E940712BE016F5F7F4F88E494E0A5
:104E80000E946E10CE0101960E94B91088E494E051
:104E90000E9448107093BE026093BD02C6CB86E3A9
:104EA00094E00E94B9108CE394E00E94B91082E46F
:104EB00094E00E94B91088E494E00E94B9108EE456
:104EC00094E00E94B91084E594E00E94B9108AE54C
:104ED00094E00E94B9108BE491E090938F0480934A
:104EE0008E048EE894E00C949E07EF920F931F932C
:104EF000CF93DF93E80134E047FD34E1042E000C4A
:104F0000550B57FF03C0519541955109E32E022FD0
:104F1000242FAE010E940828CE01DF91CF911F916E
:104F20000F91EF900895662777270C9467291F93B8
:104F3000FC0199278827BC01E89411911032E9F30C
:104F4000193010F01E30C8F31B3251F01D3249F4F5
:104F5000689406C00E94D927610F711D811D911DA3
:104F6000119110531A30B0F33EF4909580957095DE
:104F700061957F4F8F4F9F4F1F910895FB01DC017B
:104F800005900D920020E1F70895FC0105900020A6
:104F9000E9F7809590958E0F9F1F0895BB274A30A3
:104FA00031F4992322F4BDE2909581959F4F0C94A2
:104FB000EF27592F482F372F262F660F771F881F6F
:104FC000991F660F771F881F991F620F731F841F19
:104FD000951F660F771F881F991F0895BB27FB0138
:104FE0005527AA27880F991FAA1FA41710F0A41BE2
:104FF00083955051B9F7A05DAA3308F0A95DA1933C
:10500000009779F7B111B1931192CB010C94B02BA9
:10501000A9E0B0E0EEE0F8E20C94162D6A01F22E61
:10502000B02E102FFBE3AF2EA01608F41BE31F5F7A
:10503000012F27E0AE014F5F5F4F0E94B72ABC01EE
:105040008981982F9970913009F43FC09BE2E1FC6F
:1050500004C09E2D9170E0FC3AC05E2D5071E82F87
:10506000E87083FF46C084E0911101C083E0EF2D1A
:10507000E81B8F1508F0E0E0D6018E2F20E25523C3
:1050800051F1992329F0D6019C93C60101966C0138
:1050900096012D5F3F4FE2FE24C08EE4D6018C9333
:1050A00091E411969C93119712968C93D9018E2FAF
:1050B00090E281111BC0E20FF32FF11D10828EEFE1
:1050C0009FEF2996ECE00C94322D9DE2C6CF90E242
:1050D000C4CF2D9381508111FCCFCE0ED11CE0E0C6
:1050E000D0CF8EE6D6018C9391E6DBCF9D93815095
:1050F000E0CF482F447082FF3DC084E0911101C091
:1051000083E08F1510F4EF2DE81BD6018E2F20E2DF
:10511000552309F1992329F0D6019C93C6010196E4
:105120006C0196012D5F3F4FE2FE1BC089E4D60162
:105130008C938EE411968C93119786E412968C933F
:10514000D9018E2F90E2882309F4B5CF9D93815029
:10515000FACF2D9381508111FCCFCE0ED11CE0E00F
:10516000D9CF89E6D6018C938EE611968C93119750
:1051700086E6E4CF9B0177FF02C030E020E0A1E0AB
:10518000B0E0911102C0B0E0A0E0F9013196AE0F9D
:10519000BF1F8B2C912CBB2009F461C05401EFEF91
:1051A000AE1ABE0AAA0DBB1DFA161B0619F014F0A2
:1051B0004F2D4A1B511188C0E3FC59C07601A42F22
:1051C000B0E2A1114FC0C40ED11C992309F45BC0F9
:1051D00040E0D6011196F60190836D01552309F444
:1051E00048C0012F060F9A81582F507184FF03C0C9
:1051F000913309F4015010160CF047C0093008F043
:1052000008E0EEE2FE2E5B01A01AB1088501919440
:10521000819491082F3F320729F4D601FC92F601C0
:1052200031966F016217730794F1021713077CF52B
:10523000DB01A21BB30BAA24A394B12CAC0EBD1EA0
:10524000AA0DBB1D11968C9121503109D6011196E2
:1052500028153905F4F0F60180836D01DBCFB12C00
:10526000A12CA0CFF701B1937F01A150AACF91113A
:10527000B0CFD601942F50E302C05D9391509111AD
:10528000FCCFC40ED11C40E0ACCF01E0BACF80E32C
:10529000DBCF6217730731F4963388F4953311F43A
:1052A000552369F0F6018083FD01842F90E281117E
:1052B00008C0A40FB11D1C9290E080E002CF81E3F2
:1052C000F1CF91938150F3CF911183CF8ACFB0E08A
:1052D000A0E0EDE6F9E20C94162D5C017B0161156E
:1052E000710519F0DB018D939C9385010F5F1F4FB2
:1052F000F501D0818D2F90E00E948F2B6C01892BBE
:10530000B9F5DD32B9F50F5F1F4FD5011196DC916C
:10531000C1E05801F1E0AF1AB10843E050E062EF9C
:1053200070E0C5010E94982B892B69F5680182E025
:10533000C80ED11C45E050E06DEE70E0C6010E9441
:10534000982B892B21F4680197E0C90ED11CE11438
:10535000F10419F0D701CD92DC9260E070E080E8B2
:105360009FEFC111FFC060E070E080E89FE7FAC0E6
:105370005801BBCFDB3229F485010E5F1F4FF501C9
:10538000D181C0E0C6CF43E050E06AEE70E0C501D5
:105390000E94982B892BE9F0F80110E000E020E052
:1053A00030E0A9015F01B0ED8B2E8D0E89E08815EC
:1053B000C8F19C2E689491F88C2F8870C2FF16C09B
:1053C000811102C00F5F1F4F3196D501DC91C92DAD
:1053D000E9CFE114F10429F00E5F1F4FF7011183AB
:1053E000008360E070E080EC9FE7BCC0882311F090
:1053F00001501109A5E0B0E00E94FD2C9B01AC0119
:10540000220F331F441F551F280D311D411D511DF3
:10541000283999E93907490799E15907A8F2C6607F
:105420009C2ED2CFAEEF8A1206C0C3FD3CC09C2E8C
:10543000689493F8C9CFDF7DD534A9F580818D328A
:1054400039F4C061DF011296818162E070E006C02C
:10545000DF018B32C1F3119661E070E080535D0192
:10546000A61AB70A8A30F8F4E0E8CE16ECE0DE06B9
:105470005CF4B601660F771F660F771FC60ED71E46
:10548000CC0CDD1CC80ED11C5D01FFEFAF1ABF0AAA
:105490008C9180538A30A8F1C4FF03C0D194C19489
:1054A000D1080C0D1D1DC1FF09C0E114F10431F03C
:1054B00081E0A81AB108D701AD92BC92CA01B90126
:1054C0000E94C52BC370C33009F490584B015C0196
:1054D00020E030E0A9010E94C02B882309F440C0DD
:1054E000C1E2D1E017FF05C0119501951109C9E08E
:1054F000D1E06E01B8E1CB1AD10880E2E82EF12CA0
:105500000FC0D501B1CFFE01259135914591549140
:105510000E191F09C501B4010E94262C4B015C0124
:10552000D501C4010E151F0574F72497F594E7946F
:10553000CC16DD06A9F78A2F880F8B2F881F8F3F87
:1055400049F020E030E0A901C501B4010E94C02B60
:10555000811106C082E290E09093BC048093BB046A
:10556000C501B401CDB7DEB7ECE00C94322D283084
:1055700008F027E03327DA01990F311D87FD91608C
:1055800000966105710539F432602E5F3D9330E37A
:105590002A95E1F708959F3F30F080387105610545
:1055A00009F03C5F3C5F3D93913008F08068911DAD
:1055B000DF93CF931F930F93FF92EF92192F987F52
:1055C0009695E92F96959695E90FFF27E158FE4F9E
:1055D00099273327EE24FF24A701E70105900894BB
:1055E000079428F4360FE71EF81E491F511D660F59
:1055F000771F881F991F0694A1F70590079428F438
:10560000E70EF81E491F561FC11D770F881F991FEF
:10561000661F0694A1F70590079428F4F80E491F19
:10562000561FC71FD11D880F991F661F771F06942D
:10563000A1F70590079420F4490F561FC71FD81FE4
:10564000990F661F771F881F0694A9F784911095FC
:10565000177041F0D695C79557954795F794E794FD
:105660001A95C1F7E5E2F1E068941590159135912E
:105670006591959105907FE27395E118F10A430BCE
:10568000560BC90BD009C0F7E10CF11E431F561F82
:10569000C91FD01D7EF4703311F48A95E6CFE894CB
:1056A000015030F0080F0AF40027021708F4202FE9
:1056B0002395022F7A3328F079E37D932A95E9F731
:1056C00010C07D932A9589F606949795679537952E
:1056D00017951794E118F10A430B560BC90BD00923
:1056E00098F023957E9173957A3308F070E37C935C
:1056F0002013B8F77E9170617D9330F0839571E34C
:105700007D9370E32A95E1F71124EF90FF900F91BC
:105710001F91CF91DF91992787FD90950895911161
:105720000C94932C803219F089508550C8F7089555
:10573000FB01DC014150504088F08D9181341CF018
:105740008B350CF4805E659161341CF06B350CF484
:10575000605E861B611171F3990B0895881BFCCF65
:10576000DC01FC01672F71917723E1F7329704C0C8
:105770007C916D9370836291AE17BF07C8F3089553
:105780000E94022C08F481E00895E89409C097FB78
:105790003EF490958095709561957F4F8F4F9F4F08
:1057A0009923A9F0F92F96E9BB279395F69587954C
:1057B00077956795B795F111F8CFFAF4BB0F11F40F
:1057C00060FF1BC06F5F7F4F8F4F9F4F16C08823B6
:1057D00011F096E911C0772321F09EE8872F762FEC
:1057E00005C0662371F096E8862F70E060E02AF02D
:1057F0009A95660F771F881FDAF7880F9695879519
:1058000097F90895990F0008550FAA0BE0E8FEEFED
:1058100016161706E807F907C0F012161306E40774
:10582000F50798F0621B730B840B950B39F40A266D
:1058300061F0232B242B252B21F408950A2609F44B
:10584000A140A6958FEF811D811D08950E94392CDE
:105850000C94AD2C0E949F2C38F00E94A62C20F0B6
:10586000952311F00C94962C0C949C2C11240C94E0
:10587000E12C0E94BE2C70F3959FC1F3950F50E070
:10588000551F629FF001729FBB27F00DB11D639FF2
:10589000AA27F00DB11DAA1F649F6627B00DA11D98
:1058A000661F829F2227B00DA11D621F739FB00D3E
:1058B000A11D621F839FA00D611D221F749F3327AE
:1058C000A00D611D231F849F600D211D822F762F47
:1058D0006A2F11249F5750409AF0F1F088234AF024
:1058E000EE0FFF1FBB1F661F771F881F9150504090
:1058F000A9F79E3F510580F00C94962C0C94E12C56
:105900005F3FE4F3983ED4F3869577956795B79516
:10591000F795E7959F5FC1F7FE2B880F911D969530
:10592000879597F9089599278827089597F99F678C
:1059300080E870E060E008959FEF80EC0895002417
:105940000A941616170618060906089500240A94E4
:1059500012161306140605060895092E0394000C6A
:1059600011F4882352F0BB0F40F4BF2B11F460FFF9
:1059700004C06F5F7F4F8F4F9F4F089557FD905822
:10598000440F551F59F05F3F71F04795880F97FB03
:10599000991F61F09F3F79F08795089512161306BD
:1059A0001406551FF2CF4695F1DF08C016161706EC
:1059B0001806991FF1CF8695710561050894089521
:1059C000E894BB2766277727CB0197F90895F999C3
:1059D000FECF92BD81BDF89A992780B50895262FF4
:1059E000F999FECF1FBA92BD81BD20BD0FB6F894C4
:1059F000FA9AF99A0FBE019608950E94692DA59F03
:105A0000900DB49F900DA49F800D911D11240895B9
:105A1000B7FF0C94FD2C0E94FD2C821B930B089564
:105A20002F923F924F925F926F927F928F929F92AE
:105A3000AF92BF92CF92DF92EF92FF920F931F939C
:105A4000CF93DF93CDB7DEB7CA1BDB0B0FB6F8944D
:105A5000DEBF0FBECDBF09942A88398848885F848D
:105A60006E847D848C849B84AA84B984C884DF80FE
:105A7000EE80FD800C811B81AA81B981CE0FD11DE2
:105A80000FB6F894DEBF0FBECDBFED010895A1E2C1
:105A90001A2EAA1BBB1BFD010DC0AA1FBB1FEE1FA8
:105AA000FF1FA217B307E407F50720F0A21BB30BF3
:105AB000E40BF50B661F771F881F991F1A9469F76F
:105AC00060957095809590959B01AC01BD01CF01CB
:105AD0000895A29FB001B39FC001A39F700D811DC7
:105AE0001124911DB29F700D811D1124911D0895E7
:105AF0005058BB27AA270E94902D0C94AD2C0E94D1
:105B00009F2C38F00E94A62C20F039F49F3F19F406
:105B100026F40C949C2C0EF4E095E7FB0C94962C48
:105B2000E92F0E94BE2C58F3BA1762077307840747
:105B3000950720F079F4A6F50C94E02C0EF4E0958E
:105B40000B2EBA2FA02D0B01B90190010C01CA0137
:105B5000A0011124FF27591B99F0593F50F4503EE2
:105B600068F11A16F040A22F232F342F4427585FD4
:105B7000F3CF469537952795A795F0405395C9F7EC
:105B80007EF41F16BA0B620B730B840BBAF09150A4
:105B9000A1F0FF0FBB1F661F771F881FC2F70EC043
:105BA000BA0F621F731F841F48F487957795679516
:105BB000B795F7959E3F08F0B0CF9395880F08F002
:105BC0009927EE0F9795879508950E94F92D0C94CB
:105BD000AD2C0E94A62C58F00E949F2C40F029F476
:105BE0005F3F29F00C94962C51110C94E12C0C94ED
:105BF0009C2C0E94BE2C68F39923B1F3552391F39A
:105C0000951B550BBB27AA2762177307840738F02B
:105C10009F5F5F4F220F331F441FAA1FA9F335D088
:105C20000E2E3AF0E0E832D091505040E695001C3C
:105C3000CAF72BD0FE2F29D0660F771F881FBB1FF6
:105C4000261737074807AB07B0E809F0BB0B802DD4
:105C5000BF01FF2793585F4F3AF09E3F510578F000
:105C60000C94962C0C94E12C5F3FE4F3983ED4F313
:105C7000869577956795B795F7959F5FC9F7880FD4
:105C8000911D9695879597F90895E1E0660F771F26
:105C9000881FBB1F621773078407BA0720F0621BB7
:105CA000730B840BBA0BEE1F88F7E09508950E94E2
:105CB0005E2E6894B1110C94E12C08950E94C62CBC
:105CC00088F09F5798F0B92F9927B751B0F0E1F0BD
:105CD000660F771F881F991F1AF0BA95C9F714C06D
:105CE000B13091F00E94E02CB1E008950C94E02CCA
:105CF000672F782F8827B85F39F0B93FCCF38695A6
:105D000077956795B395D9F73EF490958095709502
:105D100061957F4F8F4F9F4F089597FB16F40E9418
:105D2000D12E0C94942EE894F92F96EBFF2381F05A
:105D3000121613061406440B9395F69587957795DE
:105D4000679557954040FF23B9F71BC099270895E1
:105D5000882351F49850D2F7872B762F652F542F34
:105D6000432F322F20E0B1F3121613061406440B12
:105D700088233AF09A95440F551F661F771F881F96
:105D8000CAF755234AF4440F551F11F460FF04C0AD
:105D90006F5F7F4F8F4F9F4F880F9695879597F92D
:105DA00008959095809570956095509540953095A3
:105DB00021953F4F4F4F5F4F6F4F7F4F8F4F9F4FFB
:105DC00008950E94022C08F48FEF0895FA01EE0F57
:105DD000FF1F309621053105A1F16115710561F4B0
:105DE0008038BFE39B0749F168949038810561F0E2
:105DF0008038BFEF9B0741F099234AF5FF3FE1054B
:105E00003105210519F1E8940894E795D901AA23F1
:105E100029F4AB2FBE2FF85FD0F310C0FF5F70F4F2
:105E2000A695E0F7F73950F019F0FF3A38F49F776C
:105E30009F930DD00F9007FC9058089546F00C9456
:105E40009C2C60E070E080E89FE308954FE79F7727
:105E50005F934F933F932F930E94E62F2F913F9193
:105E60004F915F910E94262C0C94432F0E94022C8C
:105E7000880B990B089529F416F00C94962C0C9429
:105E8000E02C0C949C2C0E94C62CA8F39638A0F70A
:105E900007F80F92E8942BE33AEA48EB5FE70E9499
:105EA0003C2C0F920F920F924DB75EB70F920E944B
:105EB0002E30E8E6F0E00E94752F4F915F91EF9150
:105EC000FF91E595EE1FFF1F49F0FE57E06844275C
:105ED000EE0F441FFA95E1F74195550B0E94A82F4C
:105EE0000F9007FE0C949C2F0895DF93CF931F9380
:105EF0000F93FF92EF92DF927B018C01689406C0B2
:105F0000DA2EEF010E94392CFE01E894A59125912B
:105F1000359145915591A6F3EF010E94902DFE0118
:105F20009701A801DA9469F7DF90EF90FF900F9145
:105F30001F91CF91DF9108959B01AC0160E070E06B
:105F400080E89FE30C94E52D0C94962C0C94623021
:105F50000E94C62CD8F39923C9F3940F511DA3F3C3
:105F60009150504094F059F0882332F0660F771F1B
:105F7000881F91505040C1F79E3F51052CF7880F64
:105F8000911D9695879597F908955F3FACF0983EDF
:105F90009CF0BB27869577956795B79508F4B16017
:105FA0009395C1F7BB0F58F711F460FFE8CF6F5F0F
:105FB0007F4F8F4F9F4FE3CF0C94E12C16F00C9442
:105FC00062300C949C2C68940C94962C0E94C62CE5
:105FD000A8F39923C1F3AEF3DF93CF931F930F93ED
:105FE000FF92C92FDD2788232AF02197660F771F9C
:105FF000881FDAF720E030E040E85FEB9FE3883964
:1060000020F0803E38F021968F770E94792DE0E9CC
:10601000F0E004C00E94792DEDEBF0E00E94752FB6
:106020008B01BE01EC01FB2E6F5771097595771F2F
:10603000880B990B0E94C72B28E132E741E35FE30D
:106040000E94392CAF2D9801AE01FF900F911F9146
:10605000CF91DF910E94902D0C94AD2CFA01DC01C0
:10606000AA0FBB1F9B01AC01BF5728F4222733277F
:106070004427507820C0B75190F4AB2F00244695A8
:1060800037952795011CA395D2F3002071F0220FBC
:10609000331F441FB395DAF30ED00C94782D613082
:1060A0007105A0E88A07B94630F49B01AC01662768
:1060B000772788279078309621F020833183428398
:1060C000538308959F3F31F0915020F48795779541
:1060D0006795B795880F911D9695879597F90895BF
:1060E000DB018F939F930E94FD2CBF91AF91A29FE4
:1060F000800D911DA39F900DB29F900D11240895C6
:10610000AA1BBB1B51E107C0AA1FBB1FA617B707DD
:1061100010F0A61BB70B881F991F5A95A9F78095F9
:106120009095BC01CD01089597FB072E16F40094BD
:1061300007D077FD09D00E94803007FC05D03EF4DF
:10614000909581959F4F0895709561957F4F089523
:10615000DF93CF931F930F939A9DF02D219FF00D06
:106160008B9DF00D8A9DE02DF10D039FF00D029F98
:10617000E00DF11D4E9DE00DF11D5E9DF00D4F9D5A
:10618000F00D7F936F93BF92AF925F934F93D501C2
:106190000E94692D8B01AC01D7010E94692DEB0192
:1061A000E80FF91FD6010E94F7302F913F91D601D9
:1061B0000E94692DC60FD71FE81FF91FAF91BF912D
:1061C0000E94F7302F913F910E94692DC60FD71F73
:1061D000E81FF91FD6010E94692DE60FF71F9801ED
:1061E000BE01CF010F911F91CF91DF9108950E94C1
:1061F000692D460F571FC81FD91F08F431960895FF
:10620000689401C0E894F92FF12B12F00C9434310A
:10621000A0E0B0E0EEE0F1E30C94162D092E059419
:1062200022F40E949031112392F4F0E80F26FFEF40
:10623000E094F09400951095B094C094D094A194FB
:10624000BF0ACF0ADF0AEF0AFF0A0F0B1F0B0E94DB
:106250003F3107FC0E949031CDB7DEB7ECE00C94E3
:10626000322D689401C0E8948F929F92CF93DF9370
:106270000E943F31DF91CF919F908F9008958824A5
:106280009924F401E401B0E49F93AA279A158B04A2
:106290009C04ED05FE05CF05D007A10798F4AD2FAE
:1062A000DC2FCF2FFE2FE92D982C892E982F872FAA
:1062B000762F652F542F432F322F2227B85031F7D6
:1062C000BF9127C01B2EBF91BB27220F331F441F36
:1062D000551F661F771F881F991F881C991CEE1F6A
:1062E000FF1FCC1FDD1FAA1FBB1F8A149B04EC05D8
:1062F000FD05CE05DF05A007B10748F08A189B0809
:10630000EC09FD09CE09DF09A00BB10B21601A943D
:10631000E1F62EF49401AF01BE01CD01000C089509
:106320006095709580959095309540955095219504
:106330003F4F4F4F5F4F6F4F7F4F8F4F9F4F08958E
:10634000002E083090F0982F872F762F652F542F2E
:10635000432F322F22270850F4CF220F331F441F20
:10636000551F661F771F881F991F0A95B2F7002DCA
:10637000089597FD1094002E083098F00850232FB0
:10638000342F452F562F672F782F892F912DF4CF3B
:106390001594979587957795679557954795379570
:1063A00027950A95AAF71124002D08952A0D3B1D63
:1063B0004C1D5D1D6E1D7F1D801F911F08952A19A4
:1063C0003B094C095D096E097F09800B910B08950B
:1063D0000024A7FD00942A173005400550056005EC
:1063E0007005800590050895EE0FFF1F0590F4914C
:1063F000E02D09940F931F93CF93DF938230910583
:1064000010F482E090E0E091BF04F091C00430E02D
:1064100020E0B0E0A0E0309799F42115310509F4AF
:106420004AC0281B390B24303105D8F58A819B815D
:106430006115710589F1FB0193838283FE0111C00F
:10644000408151810281138148175907E0F04817B4
:10645000590799F4109761F012960C9312971396BE
:106460001C933296CF01DF91CF911F910F91089528
:106470000093BF041093C004F4CF2115310551F0EF
:106480004217530738F0A901DB019A01BD01DF0172
:10649000F801C1CFEF01F9CF9093C0048093BF04FE
:1064A000CDCFFE01E20FF31F81939193225031096A
:1064B00039832883D7CF2091BD043091BE04232B8C
:1064C00041F420911001309111013093BE042093CA
:1064D000BD0420910E0130910F012115310541F4C9
:1064E0002DB73EB74091120150911301241B350B7B
:1064F000E091BD04F091BE04E217F307A0F42E1B57
:106500003F0B2817390778F0AC014E5F5F4F241717
:10651000350748F04E0F5F1F5093BE044093BD04F3
:10652000819391939FCFF0E0E0E09CCFCF93DF93F6
:106530000097E9F0FC01329713821282A091BF0408
:10654000B091C004ED0130E020E01097A1F420816B
:106550003181820F931F2091BD043091BE04281712
:10656000390709F061C0F093BE04E093BD04DF91E8
:10657000CF910895EA01CE17DF07E8F54A815B81E4
:106580009E0141155105B1F7E901FB83EA83499169
:106590005991C40FD51FEC17FD0761F480819181DB
:1065A0000296840F951FE9019983888382819381E4
:1065B0009B838A83F0E0E0E012968D919C91139783
:1065C0000097B9F52D913C911197CD010296820F5C
:1065D000931F2091BD043091BE042817390739F666
:1065E000309751F51092C0041092BF04B093BE04CE
:1065F000A093BD04BCCFD383C28340815181840F5B
:10660000951FC817D90761F44E5F5F4F8881998144
:10661000480F591F518340838A819B8193838283D2
:106620002115310509F0B0CFF093C004E093BF0409
:106630009ECFFD01DC01C0CF13821282D7CFB0E024
:10664000A0E0E5E2F3E30C94122D8C01009751F4E5
:10665000CB010E94FA318C01C801CDB7DEB7E0E171
:106660000C942E2DFC01E60FF71F9C0122503109DE
:10667000E217F30708F49DC0D901CD91DC91119781
:10668000C617D70798F0C530D10530F3CE0104976F
:106690008617970708F3C61BD70B2297C193D19390
:1066A0006D937C93CF010E949632D6CF5B01AC1ADA
:1066B000BD0A4C018C0E9D1EA091BF04B091C00478
:1066C000512C412CF12CE12C109731F58091BD0417
:1066D0009091BE048815990509F05CC046165706CE
:1066E00008F058C080910E0190910F01009741F47D
:1066F0008DB79EB74091120150911301841B950BE9
:10670000E817F90708F055C0F093BE04E093BD0404
:10671000F90171836083A0CF8D919C91119712969E
:106720006C90129713967C901397A815B90559F59C
:106730006C0142E0C40ED11CCA14DB0420F1AC0190
:106740004A195B09DA011296159780F0628273820A
:1067500051834083D9016D937C93E114F10471F06E
:10676000D7011396FC93EE93129776CF22968C0F57
:106770009D1FF90191838083F301EFCFF093C00453
:10678000E093BF0469CF4816590608F42C017D0137
:10679000D3019ACFCB010E94FA317C01009749F0D6
:1067A000AE01B8010E94E433C8010E94963287010D
:1067B00053CF10E000E050CF9111089581568A51D7
:1067C00008F4805285580895FB01DC0102C0019055
:1067D0000D9241505040D8F70895FB01DC01019023
:1067E0000D920020E1F70895FB01DC01415050407B
:1067F00030F08D910190801919F40020B9F7881BB1
:10680000990B0895FB01DC014150504048F0019084
:106810000D920020C9F701C01D9241505040E0F791
:10682000089511E0C1EED1E004C0FE010E94F431F0
:106830002196C23ED107C9F7F894FFCF0101640049
:1068400016000000A0400000F0410000C1048000DC
:106850005E00BC007701FF018600000000007900A7
:10686000000000C8020F0255021503860264027878
:106870000200000000D20AA50A010BD6069E0A8B70
:106880000A7C0A00000000D7060F02010BD606336F
:10689000074B07BE060D0A00543D006F4320004819
:1068A0003D0025006F4320413D0054003D4E6F20C8
:1068B00053656E736F7221005428312C322C3329AA
:1068C0003D00206F4320445320546865726D6F6D06
:1068D000657465720055563D00434F323D0070703F
:1068E0006D003A00504D28312E302C322E352C318F
:1068F00030293D00206E672F4C004C3D00206C7805
:106900002000424E4D4C3033004E616E6F42326279
:10691000330073657269616C3A20002D35002D34A7
:10692000002D33002D32002D310044005665727366
:10693000696F6E3A200023007300534C20503D00D5
:10694000506120697320756E6C696B656C792100EC
:10695000536561206C6576656C20503D0020685061
:0A696000610055565A005620000051
:107E0000112484B714BE81FFF0D085E080938100F7
:107E100082E08093C00088E18093C10086E0809377
:107E2000C20080E18093C4008EE0C9D0259A86E02C
:107E300020E33CEF91E0309385002093840096BBD3
:107E4000B09BFECF1D9AA8958150A9F7CC24DD24C4
:107E500088248394B5E0AB2EA1E19A2EF3E0BF2EE7
:107E6000A2D0813461F49FD0082FAFD0023811F036
:107E7000013811F484E001C083E08DD089C08234E0
:107E800011F484E103C0853419F485E0A6D080C0E4
:107E9000853579F488D0E82EFF2485D0082F10E0AE
:107EA000102F00270E291F29000F111F8ED06801E7
:107EB0006FC0863521F484E090D080E0DECF843638
:107EC00009F040C070D06FD0082F6DD080E0C81688
:107ED00080E7D80618F4F601B7BEE895C0E0D1E017
:107EE00062D089930C17E1F7F0E0CF16F0E7DF06D8
:107EF00018F0F601B7BEE89568D007B600FCFDCFD4
:107F0000A601A0E0B1E02C9130E011968C91119780
:107F100090E0982F8827822B932B1296FA010C0160
:107F200087BEE89511244E5F5F4FF1E0A038BF0790
:107F300051F7F601A7BEE89507B600FCFDCF97BE46
:107F4000E89526C08437B1F42ED02DD0F82E2BD052
:107F50003CD0F601EF2C8F010F5F1F4F84911BD097
:107F6000EA94F801C1F70894C11CD11CFA94CF0C13
:107F7000D11C0EC0853739F428D08EE10CD085E9AC
:107F80000AD08FE07ACF813511F488E018D01DD067
:107F900080E101D065CF982F8091C00085FFFCCF94
:107FA0009093C60008958091C00087FFFCCF809118
:107FB000C00084FD01C0A8958091C6000895E0E648
:107FC000F0E098E1908380830895EDDF803219F02E
:107FD00088E0F5DFFFCF84E1DECF1F93182FE3DFCA
:107FE0001150E9F7F2DF1F91089580E0E8DFEE27F6
:047FF000FF270994CA
:027FFE00040479
:00000001FF
